:020000040000fa
:080000000002040000000000f2
:020000040000fa
:10000800d2020000d2020000d2020000d202000098
:10001800d2020000d2020000d2020000d202000088
:10002800d2020000d2020000d2020000d202000078
:10003800d2020000d2020000d2020000d202000068
:020000040000fa
:020000040000fa
:100400006fe621000ebf25000e01880000000000ed
:10041000000020000000e000020032000001200087
:10042000200288000c000700a0a626000100200082
:100430000f000700000020000000e0000200320072
:100440000000020000000000ca6802000000000076
:100450000040da000000fe00000420000000e00080
:1004600002003200002020009001880000000600f9
:10047000a1028800800078000000eb001a0037001d
:10048000e280400054a0b4009101ba00e280400034
:1004900054a0b4009102ba00e280400054a0b4001d
:1004a0000002eb00472bde00f507b200a601880032
:1004b000602ce10008003a000049eb000201e8006e
:1004c000020039003420ec0002f0a0008301e900b2
:1004d000f9ff3e00040037006128e100010032000e
:1004e0000082eb00040007001101ba000200e000e6
:1004f000e3ff3a000000060004d0a300e20f490029
:100500001c003900810278003549ba000201e80078
:10051000020039003420ec0002f0a0008301e90061
:100520000f0032002549ba000201e800020039003c
:100530003420ec0002f0a0008301e9000800320042
:100540000400e0000600320015c9ba000201e8000c
:10055000020039003420ec0002f0a0008301e90021
:100560008180e80054a0b4000300e000e2ff3a00fc
:10057000000006009102ba00055978008301e900e5
:10058000f7ff3200c82ade00055978008301e90030
:10059000f3ff32000400e000f1ff320011d9ba008d
:1005a000eeff37000040da000000fe0003f0a2007a
:1005b000889fbe008a9fbe008c1f7800f60007004f
:1005c000fd0033006450e1004f0032006420e10080
:1005d0005200320003826c0007003b000905d00086
:1005e0000306d000820f54000c065d0002003900a3
:1005f00002003200890178000306780085825500e8
:1006000004003d000003fd008103fd008502ea00b7
:100610008b854200840f720002003b0060001000d6
:10062000e08018006011b8000005eb007a28e100b6
:100630000a00390006007800c75ddd00f707b20048
:10064000878075002d003700828171000a017800d3
:10065000610560008180d1000080d3008502e9003f
:10066000f9ff3b00060440008784480002003b007d
:1006700060041400e0841c000988a3000700320015
:100680008a81710082817100610164008904d10056
:100690000884d3008b05e800170037000978a30011
:1006a00013003a000b00e000130034008b05e90052
:1006b0000804440089844c000a4474000978a300ab
:1006c0000d003a000b00e000070034008b05e90044
:1006d0000804440089844c0001003a000b0020000b
:1006e0000978a300f7ff32000001eb000200370099
:1006f000828171000a0178006c0007000cf0a700ed
:1007000001f0a000b50037006420e10002003a00cb
:10071000838f6c00b50033000801be000200be00ec
:10072000ae003700889fbe008a9fbe008c1f7800f5
:1007300099000700a000330003866c006450e100bc
:100740002e0032006420e100330032006150e100ed
:100750002f0032006120e100310032008585550014
:10076000eb07b00009002000080420000500370056
:100770000804440089844c000a0031000603430049
:1007800087834b000001530081815b00f8ff330039
:100790000203be000800a0000804440089844c0045
:1007a000f6ff3900c639dd00830173000100320015
:1007b000130020008904d1000884d3000998a30005
:1007c000050032000800a7000300a0008904d10042
:1007d0000884d3008b05e8008904d1000884d30085
:1007e0000001eb000281d2003000070001f0a100ff
:1007f0000cf0a70001f0a000780037006420e100b1
:100800007a0032000801be000200be00f7ff370088
:100810006120e100750032006000b800f3ff37008e
:100820000000200001f82700f0ff37000001be00a3
:10083000440007000470a70003f0a10003f8a30020
:1008400013003a006509b1001000320009003500bc
:100850006928e100020035000100280000000500c1
:1008600000004000818048008502e900fcff3a005a
:1008700000000600f88f4200050035008100d1001d
:100880000080d3008502e800fcff3a00000006006b
:100890008000eb00000005004f89de008201780037
:1008a0008b0037006011b8009900370081002000ec
:1008b000618055000b003d000b00200061fe2f0001
:1008c0000100e1001d0034008281710061016400bb
:1008d0008904d1000884d3000000e800faff3a0040
:1008e00071002000610064000300700002006000dd
:1008f0000900320061044400e0844c000988a5002e
:10090000050032008b05e8006808e10002003a00ab
:100910008904d1000884d300f20f20000258e100be
:1009200005003d00c75ddd00f907b2008980750054
:1009300008007800000006000bf827008b00780004
:1009400000000500c70ade00f107b200f50fb20093
:1009500008003200e1cf4200020032000170a00026
:1009600024000500810f700001003200040805001a
:1009700044000500810f700002003a0014000500d9
:100980008502e9000000400081c04800fcff3b00f8
:100990000170a000240005000004be00e9ff07006c
:1009a0000003be000405be000200be00e5ff070014
:1009b000844f7500000006000200be006450e10094
:1009c000050036006420e100020036000968a3003b
:1009d00001003a000800be000160a0004f06780048
:1009e0004f05be004f04be0000000600f0ff2f00c0
:1009f000f1ff2700f9ff3700889fbe008a9fbe00e5
:100a00008c1f7800e4ff0700ebff330003866c00c7
:100a10006450e100240032006420e100270032002d
:100a20006150e100220032006120e100210032002b
:100a30008b854200eb07b1000134b800003ab800e2
:100a40000804420089844a00013ab8000030b80026
:100a50008880400009014a00040033000000400083
:100a600081804800020149008b05e900c909dd00c9
:100a7000830170000100320013002000c814de0062
:100a80004814dd004709de001200b200c808de008d
:100a90000884700085ff070001f0a1000cf0a7009a
:100aa00001f0a000cdff37006120e100cfff320050
:100ab0000801be000200be00f7ff37006150e100f0
:100ac000fcff3a00c9ff37000001eb003f00370090
:100ad000881f7800030478000300e00007003d0051
:100ae00060001000e080180060011900e08119002a
:100af00002003b0001f02d00030037000400070056
:100b000008f0a70001f0a0004f04780000000600e4
:100b1000889fbe008a9fbe000082700004027100a0
:100b200004827100260032000004be000200be00f4
:100b30006011b8006b092000950220000182cf00ef
:100b40000a0039000541b1000082cf0007003900da
:100b50000541b1000982cf00040039000541b10010
:100b60000882cf00010039000541b1000542520062
:100b7000120032000a003b008281710061016400b2
:100b80008100d1000080d3008984d3000884d30081
:100b90008b05e8000442e800f7ff3a000700370041
:100ba0000804440089844c0000004800818048000b
:100bb0008b05e9000442e900f9ff3a003bff07001a
:100bc0004f05be004f04be0000000600889fbe0017
:100bd0008a9fbe008c9fbe00820578000004be0084
:100be00058ff07000800be006420e100070039003c
:100bf00002003a00f1ff2700f0ff2f000160a00083
:100c00001202200022f38800550037006120e10025
:100c100003003a000b00a70001f823005000370042
:100c200001f0a1000200210093642400500007009d
:100c30000800be0004003500b2fd2000930c240023
:100c40006e0007000004be000005eb000b00a600cc
:100c50004f0dde0001f0a1000004be0032982f000d
:100c600023ea230064ff07000001eb0003f02300e8
:100c70000b00a70003f823004dfe07003e0007000d
:100c80000000a7000a00a20003ff07000b00e0001d
:100c9000030032000200200003f0230043fe07009f
:100ca00001f0a2000006be00020020009304240010
:100cb00051ff07000801be003dfe0700809fbe00f7
:100cc0000c00be0022a22a00d3a723004aff07007f
:100cd0004f01be0036fe07000004be0001f0a10077
:100ce0000200200003982300210007000800be0036
:100cf000190035000001be003fff07000006be00de
:100d0000b2c52900e36223003bff070022222b002b
:100d1000f3942b0026fe07000c01be0036ff0700ef
:100d2000e273280083c0230021fe07000c01be00ef
:100d300031ff070042aa2a00a3e22b001cfe070095
:100d40000c01be002cff07000801be002aff0700af
:100d50000801be0016fe07000a00a70001f0a2006d
:100d60004f06be004f05be004f04be000000060047
:100d700014002000720037000001be00f1fe0700e1
:100d80000470a70003f0a1006509b100160032004d
:100d90000d0035006828e10006003500f0ff2f0047
:100da000f1ff27000300e00013003b0001002800d2
:100db0000000050000004000818048008502e90035
:100dc000fcff3a0008003700f88f420002003c00a8
:100dd0008000eb00000005008100d1000080d300fe
:100de0008502e800fcff3a000300e00002003b003f
:100df00060001000e08018000000060004002000e1
:100e000000003700889fbe008a9fbe008c1f7800bc
:100e10004f26dd00e0fe0700e7fe33006120e10021
:100e2000430032006250e10041003e003e003900c4
:100e30006420e1003c003200058255000f003b00b9
:100e40000402e80038003a00800f5300818f5b00f5
:100e5000350034000800be0003f0a10001f0a60038
:100e600003f0a0000cf0a700d1fd0700dbfe370067
:100e70000603430087834b000c46460000055300e1
:100e800081855b00020033000a03be000c00a00055
:100e90000402e900f6ff3b008505780006024300e6
:100ea00087824b0004003a006000b80009f0a700f8
:100eb00001f0a000c9fe37000002520081825a00f2
:100ec0000704e000040033000603430087834b005f
:100ed0008b05e900faff3700090578000604be001b
:100ee0000203be006011b80070fe0700e00f520060
:100ef000e08f5a000700350002003c000c08a300f8
:100f0000040032000601be0003f0a0000cf0a700b0
:100f1000a7fd07000a85680001f0a1000af0a700fc
:100f200001f0a000adfe37000800be00abfe3700a8
:100f3000100220000cf0a60020f38800abfe370062
:100f4000889fbe008a9fbe00841f780092fe070023
:100f50004f00780011003300f0ff2f00838f6c00ea
:100f600006003b00040565000a00a70008003700e2
:100f700009f0a6001000200008003700820f54007e
:100f8000838f5c00030039001000200001003e0048
:100f90000000200009f0a7000000ea004f05be0095
:0c0fa0004f04be000000e000000006004e
:020000040000fa
:100fac00d3000000f7000000ff000000e900000083
:100fbc00a300000076000000fd0000006f000000a0
:100fcc00db000000fb00000093000000fb000000b1
:100fdc00ff000000bf000000fd000000fe0000004c
:100fec00510000005d0000003f000000d300000035
:100ffc00ab0000009700000093000000830000008d
:10100c0021000000290000004d0000002500000018
:10101c006b00000063000000ff000000f700000000
:020000040000fa
:10102c000000fa00889fbe008a9fbe008c9fbe0005
:10103c004487a8003d3a8000fc1f20008c86660087
:10104c000cc025000d0676003c3a88000ac025002d
:10105c000b0020000a057800ca38880008c025005b
:10106c000900200008047800d838880002c0250048
:10107c0003002000020178006238880000c02500bf
:10108c0001002000000078007038880006c02500a0
:10109c0007002000060378008638880004c025006d
:1010ac000500200004027800943888000082eb00d0
:1010bc00f4398800243980000400a0000410a10039
:1010cc000420a100243988000082eb00f439880048
:1010dc00a538800004802f0084826200040a20005e
:1010ec0005027200a4388800a5388000f47f200027
:1010fc0084826200f47f200004826200e638800063
:10110c0005802f008502630005027200e438880018
:10111c00b538800004802f0084826200041e2000f9
:10112c0005027200b4388800b5388000f47f2000c6
:10113c0084826200f47f200004826200f638800012
:10114c0005802f008502630005027200f4388800c8
:10115c000539800004802f0084826200840f2000f7
:10116c0005027200043988001539800004802f00b4
:10117c0084826200941f20000502720014398800da
:10118c0026e7a9002647a90026c7a9002627a800fc
:10119c002607a80026a7a9002687a90084c1b300aa
:1011ac00040078002fe7b700f47220001442780096
:1011bc000400780029e7b70084c5b3000400780068
:1011cc002ee7b700e4722000144278000400780087
:1011dc0028e7b700a4c0b300040078002ce7b700e0
:1011ec0004c2b300040078002ae7b70054c0b3006f
:1011fc00040078002de7b70084c1b3000400780028
:10120c002be7b7002667a9002727a8002707a80007
:10121c00243880000450a0000460a0000470a100d9
:10122c0024388800243880004522de0067426200a2
:10123c000482fb00670262004522dd002639800033
:10124c00f5f12f0085026300050272002439880035
:10125c0005e7a80000e8230001002000c9320700c0
:10126c0004002800843988004f06be004f05be00dc
:10127c004f04be000080fa00000006000200fa00d5
:10128c00000f780000000000010037000000000093
:10129c003438800062026200e00f5200fbff3a001b
:1012ac001e02780004388800046026001438880078
:1012bc00000000000080fa00000006000400fa00a4
:1012cc00008fbe000000000001003700000000008d
:1012dc003438800061026200e00f5200fbff3200e4
:1012ec001e02be0004027800843888001e02be0074
:1012fc0004027800943888000080fa000000060090
:10130c000400fa00008fbe001e02be00040278002a
:10131c00c43888001e02be0004027800d43888004d
:10132c000080fa00000006000800fa00000f7800a8
:10133c00110798002207980033079800000000005e
:10134c0001003700000000003438800062026200a7
:10135c00e00f5200fbff3a009e029000040a2000ae
:10136c0004aab900040278001e0242000438880066
:10137c001e0278006120b8001e02900005002000bb
:10138c00060a200006abb900060378006021b900fc
:10139c00820378000703430084027800040a2000cb
:1013ac00042ab800050343008602780000024200bc
:1013bc0081824a00402ade00840278000430260034
:1013cc0005027200143888000000000000000000c4
:1013dc000100370000000000343880006202620017
:1013ec00e00f5200fbff3a002e029000cc22dd00f1
:1013fc003e02900005027200043888002e02900014
:10140c00c422de0004402600050272001438880055
:10141c000000000000000000010037000000000088
:10142c003438800062026200e00f5200fbff3a0089
:10143c000406200004388800047026001438880044
:10144c00000000000080fa00000006000000fa0016
:10145c000000eb0089ff0700031e2000020a200099
:10146c008000eb000000eb00afff07000080fa00eb
:10147c00000006000400fa00000f78001107980025
:10148c001e027800044278000002fd0030e7b7002d
:10149c000002fd003107a8001e029000943988005c
:1014ac0000000000010037000000000085398000ba
:1014bc000400240004826200e00f5200faff3a009c
:1014cc003107a9000080fa0000000600ee05fa00c2
:1014dc00889fbe008a9fbe008c9fbe00000f7800c4
:1014ec00320a20009e004100610ab800848fd200ad
:1014fc008582d2000402780004f0a10006c0250009
:10150c0007002000900180008601d0000404d00068
:10151c00088241004220a80085824b004200a900ad
:10152c004220ae004200a8000482d30005037800dc
:10153c00960188000402780014427800900188001b
:10154c000440e800610ab800848fd2008582d20082
:10155c000402780004f0a10002c025000300200062
:10156c008204d0008400d000018244004220a800f4
:10157c00858249004200a9004220ae004200a8002a
:10158c000482d300a70180000503780004027800d0
:10159c00a6018800004a7800a7018800420a2000b2
:1015ac009e004100610ab800848fd2008582d2006f
:1015bc000402780004f0a10008c0250009002000f6
:1015cc00970180008801d0000403d00006824100fe
:1015dc004220a80085824c004200a9004220ae00a7
:1015ec004200a8000482d30005037800960188000d
:1015fc000402780014427800970188000440e80047
:10160c00610ab800848fd2008582d200040278006f
:10161c0004f0a1000ac025000b0020008a03d000b2
:10162c000404d000088243004220a80085824d00ab
:10163c004200a9004220ae004200a8000482d30060
:10164c00a70180000503780004027800a601880039
:10165c00004a7800a7018800291420009e804400cd
:10166c00610ab800848fd2008582d200040278000f
:10167c0004f0a1000cc025000d0020009701800093
:10168c000c01d0008401d000030241004220a800cc
:10169c0085824e004200a9004220ae004200a80004
:1016ac000482d300050378009601880004027800b8
:1016bc0014427800970188000440e800610ab800e1
:1016cc00848fd2008582d2000402780004f0a1003d
:1016dc0006c0250016079800070020002707980071
:1016ec001e049000ae0490008800d0000401d000cd
:1016fc00028240004220a80085824c004200a900d2
:10170c004220ae004200a8000482d300a701800052
:10171c000503780004027800a6018800004a7800ce
:10172c00a7018800331420009e804100610ab80094
:10173c00848fd2008582d2000402780004f0a100cc
:10174c0006c02500360798000700200047079800c0
:10175c00970180003e049000ce0490000801d00058
:10176c008401d000030241004220a80085824c0075
:10177c004200a9004220ae004200a8000482d3001f
:10178c000503780096018800040278001442780062
:10179c00970188000440e800610ab800848fd200e9
:1017ac008582d2000402780004f0a10006c0250056
:1017bc005607980007002000670798005e04900009
:1017cc00ee0490008800d0000401d000028240009a
:1017dc004220a80085824c004200a9004220ae00a5
:1017ec004200a8000482d300a70180000503780002
:1017fc0004027800a6018800004a7800a70188003e
:10180c00431420009e804100610ab800848fd200ee
:10181c008582d2000402780004f0a10006c02500e5
:10182c007607980007002000070f980097018000aa
:10183c007e0490008e0c90000801d0008401d00032
:10184c00030241004220a80085824c004200a900fe
:10185c004220ae004200a8000482d30005037800a9
:10186c0096018800040278001442780097018800e1
:10187c000440e800610ab800848fd2008582d2004f
:10188c000402780004f0a10006c02500160f980091
:10189c0007002000270f98001e0c9000ae0c900043
:1018ac008800d0000401d000028240004220a80031
:1018bc0085824c004200a9004220ae004200a800e4
:1018cc000482d300a701800005037800040278008d
:1018dc00a6018800004a7800a70188005314200054
:1018ec009e804100610ab800848fd2008582d200ac
:1018fc000402780004f0a10006c02500360f980001
:10190c0007002000470f9800970180003e0c9000c4
:10191c00ce0c90000801d0008401d00003024100dd
:10192c004220a80085824c004200a9004220ae0053
:10193c004200a8000482d3000503780096018800b9
:10194c000402780014427800970188000440e800f3
:10195c00610ab800848fd2008582d200040278001c
:10196c0004f0a10006c02500560f980007002000c7
:10197c00670f98005e0c9000ee0c90008800d00071
:10198c000401d000028240004220a80085824c0055
:10199c004200a9004220ae004200a8000482d300fd
:1019ac00a70180000503780004027800a6018800d6
:1019bc00004a7800a7018800231e20009e80410069
:1019cc00610ab800848fd2008582d20004027800ac
:1019dc0004f0a10006c02500760f98000700200037
:1019ec0007179800970180007e0c90008e149000d1
:1019fc000801d0008401d000030241004220a8005d
:101a0c0085824c004200a9004220ae004200a80092
:101a1c000482d30005037800960188000402780044
:101a2c0014427800970188000440e800610ab8006d
:101a3c00848fd2008582d2000402780004f0a100c9
:101a4c0006c02500161798000700200027179800dd
:101a5c001e149000ae1490008800d0000401d00039
:101a6c00028240004220a80085824c004200a9005e
:101a7c004220ae004200a8000482d300a7018000df
:101a8c000503780004027800a6018800004a78005b
:101a9c00a7018800331e20009e804100610ab80017
:101aac00848fd2008582d2000402780004f0a10059
:101abc0006c025003617980007002000471798002d
:101acc00970180003e149000ce1490000801d000c5
:101adc008401d000030241004220a80085824c0002
:101aec004200a9004220ae004200a8000482d300ac
:101afc0005037800960188000402780014427800ef
:101b0c00970188000440e800610ab800848fd20075
:101b1c008582d2000402780004f0a10006c02500e2
:101b2c005617980007002000671798005e14900065
:101b3c00ee1490008800d0000401d0000282400016
:101b4c004220a80085824c004200a9004220ae0031
:101b5c004200a8000482d300a7018000050378008e
:101b6c0004027800a6018800004a7800a7018800ca
:101b7c00431e20009e804100610ab800848fd20071
:101b8c008582d2000402780004f0a10006c0250072
:101b9c007617980007002000071f98009701800017
:101bac007e1490008e1c90000801d0008401d0009f
:101bbc00030241004220a80085824c004200a9008b
:101bcc004220ae004200a8000482d3000503780036
:101bdc00960188000402780014427800970188006e
:101bec000440e800610ab800848fd2008582d200dc
:101bfc000402780004f0a10006c02500161f98000e
:101c0c0007002000271f98001e1c9000ae1c90009f
:101c1c008800d0000401d000028240004220a800bd
:101c2c0085824c004200a9004220ae004200a80070
:101c3c000482d300a7018000050378000402780019
:101c4c00a6018800004a7800a7018800531e2000d6
:101c5c009e804100610ab800848fd2008582d20038
:101c6c000402780004f0a10006c02500361f98007d
:101c7c0007002000471f9800970180003e1c900031
:101c8c00ce1c90000801d0008401d000030241005a
:101c9c004220a80085824c004200a9004220ae00e0
:101cac004200a8000482d300050378009601880046
:101cbc000402780014427800970188000440e80080
:101ccc00610ab800848fd2008582d20004027800a9
:101cdc0004f0a10006c02500561f98000700200044
:101cec00671f98005e1c9000ee1c90008800d000ce
:101cfc000401d000028240004220a80085824c00e2
:101d0c004200a9004220ae004200a8000482d30089
:101d1c00a70180000503780004027800a601880062
:101d2c00004a7800a7018800232820009e804100eb
:101d3c00610ab800848fd2008582d2000402780038
:101d4c0004f0a10006c02500761f980007002000b3
:101d5c0007279800970180007e1c90008e2490002d
:101d6c000801d0008401d000030241004220a800e9
:101d7c0085824c004200a9004220ae004200a8001f
:101d8c000482d300050378009601880004027800d1
:101d9c0014427800970188000440e800610ab800fa
:101dac00848fd2008582d2000402780004f0a10056
:101dbc0006c025001627980007002000272798004a
:101dcc001e249000ae2490008800d0000401d000a6
:101ddc00028240004220a80085824c004200a900eb
:101dec004220ae004200a8000482d300a70180006c
:101dfc000503780004027800a6018800004a7800e8
:101e0c00a7018800332820009e804100610ab80099
:101e1c00848fd2008582d2000402780004f0a100e5
:101e2c0006c0250036279800070020004727980099
:101e3c00970180003e249000ce2490000801d00031
:101e4c008401d000030241004220a80085824c008e
:101e5c004200a9004220ae004200a8000482d30038
:101e6c00050378009601880004027800144278007b
:101e7c00970188000440e800610ab800848fd20002
:101e8c008582d2000402780004f0a10006c025006f
:101e9c005627980007002000672798005e249000c2
:101eac00ee2490008800d0000401d0000282400093
:101ebc004220a80085824c004200a9004220ae00be
:101ecc004200a8000482d300a7018000050378001b
:101edc0004027800a6018800004a7800a701880057
:101eec00432820009e804100610ab800848fd200f4
:101efc008582d2000402780004f0a10006c02500ff
:101f0c007627980007002000072f98009701800083
:101f1c007e2490008e2c90000801d0008401d0000b
:101f2c00030241004220a80085824c004200a90017
:101f3c004220ae004200a8000482d30005037800c2
:101f4c0096018800040278001442780097018800fa
:101f5c000440e800610ab800848fd2008582d20068
:101f6c000402780004f0a10006c02500162f98008a
:101f7c0007002000272f98001e2c9000ae2c9000fc
:101f8c008800d0000401d000028240004220a8004a
:101f9c0085824c004200a9004220ae004200a800fd
:101fac000482d300a70180000503780004027800a6
:101fbc00a6018800004a7800a70188005328200059
:101fcc009e804100610ab800848fd2008582d200c5
:101fdc000402780004f0a10006c02500362f9800fa
:101fec0007002000472f9800970180003e2c90009e
:101ffc00ce2c90000801d0008401d00003024100d7
:10200c004220a80085824c004200a9004220ae006c
:10201c004200a8000482d3000503780096018800d2
:10202c000402780014427800970188000440e8000c
:10203c00610ab800848fd2008582d2000402780035
:10204c0004f0a10006c02500562f980007002000c0
:10205c00672f98005e2c9000ee2c90008800d0002a
:10206c000401d000028240004220a80085824c006e
:10207c004200a9004220ae004200a8000482d30016
:10208c00a70180000503780004027800a6018800ef
:10209c00004a7800a7018800133220009e8041007e
:1020ac00610ab800848fd2008582d20004027800c5
:1020bc0004f0a10006c02500762f98000700200030
:1020cc0007379800970180007e2c90008e3490008a
:1020dc000801d0008401d000030241004220a80076
:1020ec0085824c004200a9004220ae004200a800ac
:1020fc000482d3000503780096018800040278005e
:10210c0014427800970188000440e800610ab80086
:10211c00848fd2008582d2000402780004f0a100e2
:10212c0006c02500163798000700200027379800b6
:10213c001e349000ae3490008800d0000401d00012
:10214c00028240004220a80085824c004200a90077
:10215c004220ae004200a8000482d300a7018000f8
:10216c000503780004027800a6018800004a780074
:10217c00a7018800233220009e804100610ab8002c
:10218c00848fd2008582d2000402780004f0a10072
:10219c0006c0250036379800070020004737980006
:1021ac00970180003e349000ce3490000801d0009e
:1021bc008401d000030241004220a80085824c001b
:1021cc004200a9004220ae004200a8000482d300c5
:1021dc000503780096018800040278001442780008
:1021ec00970188000440e800610ab800848fd2008f
:1021fc008582d2000402780004f0a10006c02500fc
:10220c005637980007002000673798005e3490001e
:10221c00ee3490008800d0000401d000028240000f
:10222c004220a80085824c004200a9004220ae004a
:10223c004200a8000482d300a701800005037800a7
:10224c0004027800a6018800004a7800a7018800e3
:10225c00333220009e804100610ab800848fd20086
:10226c008582d2000402780004f0a10006c025008b
:10227c007637980007002000073f980097018000f0
:10228c007e3490008e3c90000801d0008401d00078
:10229c00030241004220a80085824c004200a900a4
:1022ac004220ae004200a8000482d300050378004f
:1022bc009601880004027800144278009701880087
:1022cc000440e800610ab800848fd2008582d200f5
:1022dc000402780004f0a10006c02500163f980007
:1022ec0007002000273f98001e3c9000ae3c900059
:1022fc008800d0000401d000028240004220a800d7
:10230c0085824c004200a9004220ae004200a80089
:10231c000482d300a7018000050378000402780032
:10232c00a6018800004a7800a701880043322000eb
:10233c009e804100610ab800848fd2008582d20051
:10234c000402780004f0a10006c02500363f980076
:10235c0007002000473f9800970180003e3c90000a
:10236c00ce3c90000801d0008401d0000302410053
:10237c004220a80085824c004200a9004220ae00f9
:10238c004200a8000482d30005037800960188005f
:10239c000402780014427800970188000440e80099
:1023ac00610ab800848fd2008582d20004027800c2
:1023bc0004f0a10006c02500563f9800070020003d
:1023cc00673f98005e3c9000ee3c90008800d00087
:1023dc000401d000028240004220a80085824c00fb
:1023ec004200a9004220ae004200a8000482d300a3
:1023fc00a70180000503780004027800a60188007c
:10240c00004a7800a7018800533220009e804100ca
:10241c00610ab800848fd2008582d2000402780051
:10242c0004f0a10006c02500763f980007002000ac
:10243c0007879800970180007e3c90008e84900066
:10244c000801d0008401d000030241004220a80002
:10245c0085824c004200a9004220ae004200a80038
:10246c000482d300050378009601880004027800ea
:10247c0014427800970188000440e800610ab80013
:10248c00848fd2008582d2000402780004f0a1006f
:10249c0006c02500168798000700200027879800a3
:1024ac001e849000ae8490008800d0000401d000ff
:1024bc00028240004220a80085824c004200a90004
:1024cc004220ae004200a8000482d300a701800085
:1024dc000503780004027800a6018800004a780001
:1024ec00a7018800633220009e804100610ab80079
:1024fc00848fd2008582d2000402780004f0a100ff
:10250c0006c02500368798000700200047879800f2
:10251c00970180003e849000ce8490000801d0008a
:10252c008401d000030241004220a80085824c00a7
:10253c004200a9004220ae004200a8000482d30051
:10254c000503780096018800040278001442780094
:10255c00970188000440e800610ab800848fd2001b
:10256c008582d2000402780004f0a10006c0250088
:10257c005687980007002000678798005e849000bb
:10258c00ee8490008800d0000401d000028240004c
:10259c004220a80085824c004200a9004220ae00d7
:1025ac004200a8000482d300a70180000503780034
:1025bc0004027800a6018800004a7800a701880070
:1025cc00133c20009e804100610ab800848fd20029
:1025dc008582d2000402780004f0a10006c0250018
:1025ec007687980007002000078f980097018000dd
:1025fc007e8490008e8c90000801d0008401d00065
:10260c00030241004220a80085824c004200a90030
:10261c004220ae004200a8000482d30005037800db
:10262c009601880004027800144278009701880013
:10263c000440e800610ab800848fd2008582d20081
:10264c000402780004f0a10006c02500168f980043
:10265c0007002000278f98001e8c9000ae8c9000f5
:10266c008800d0000401d000028240004220a80063
:10267c0085824c004200a9004220ae004200a80016
:10268c000482d300a70180000503780004027800bf
:10269c00a6018800004a7800a7018800233c20008e
:1026ac009e804100610ab800848fd2008582d200de
:1026bc000402780004f0a10006c02500368f9800b3
:1026cc0007002000478f9800970180003e8c9000f7
:1026dc00ce8c90000801d0008401d0000302410090
:1026ec004220a80085824c004200a9004220ae0086
:1026fc004200a8000482d3000503780096018800ec
:10270c000402780014427800970188000440e80025
:10271c00610ab800848fd2008582d200040278004e
:10272c0004f0a10006c02500568f98000700200079
:10273c00678f98005e8c9000ee8c90008800d00023
:10274c000401d000028240004220a80085824c0087
:10275c004200a9004220ae004200a8000482d3002f
:10276c00a70180000503780004027800a601880008
:10277c00004a7800a7018800333c20009e8041006d
:10278c00610ab800848fd2008582d20004027800de
:10279c0004f0a10006c02500768f980007002000e9
:1027ac0007979800970180007e8c90008e94900083
:1027bc000801d0008401d000030241004220a8008f
:1027cc0085824c004200a9004220ae004200a800c5
:1027dc000482d30005037800960188000402780077
:1027ec0014427800970188000440e800610ab800a0
:1027fc00848fd2008582d2000402780004f0a100fc
:10280c0006c025001697980007002000279798000f
:10281c001e949000ae9490008800d0000401d0006b
:10282c00028240004220a80085824c004200a90090
:10283c004220ae004200a8000482d300a701800011
:10284c000503780004027800a6018800004a78008d
:10285c00a7018800433c20009e804100610ab8001b
:10286c00848fd2008582d2000402780004f0a1008b
:10287c0006c025003697980007002000479798005f
:10288c00970180003e949000ce9490000801d000f7
:10289c008401d000030241004220a80085824c0034
:1028ac004200a9004220ae004200a8000482d300de
:1028bc000503780096018800040278001442780021
:1028cc00970188000440e800610ab800848fd200a8
:1028dc008582d2000402780004f0a10006c0250015
:1028ec005697980007002000679798005e94900018
:1028fc00ee9490008800d0000401d00002824000c9
:10290c004220a80085824c004200a9004220ae0063
:10291c004200a8000482d300a701800005037800c0
:10292c0004027800a6018800004a7800a7018800fc
:10293c00533c20009e804100610ab800848fd20075
:10294c008582d2000402780004f0a10006c02500a4
:10295c007697980007002000079f98009701800049
:10296c007e9490008e9c90000801d0008401d000d1
:10297c00030241004220a80085824c004200a900bd
:10298c004220ae004200a8000482d3000503780068
:10299c0096018800040278001442780097018800a0
:1029ac000440e800610ab800848fd2008582d2000e
:1029bc000402780004f0a10006c02500169f9800c0
:1029cc0007002000279f98001e9c9000ae9c900052
:1029dc008800d0000401d000028240004220a800f0
:1029ec0085824c004200a9004220ae004200a800a3
:1029fc000482d300a701800005037800040278004c
:102a0c00a6018800004a7800a7018800633c2000da
:102a1c009e804100610ab800848fd2008582d2006a
:102a2c000402780004f0a10006c02500369f98002f
:102a3c0007002000479f9800970180003e9c900063
:102a4c00ce9c90000801d0008401d000030241000c
:102a5c004220a80085824c004200a9004220ae0012
:102a6c004200a8000482d300050378009601880078
:102a7c000402780014427800970188000440e800b2
:102a8c00610ab800848fd2008582d20004027800db
:102a9c0004f0a10006c02500569f980007002000f6
:102aac00679f98005e9c9000ee9c90008800d00080
:102abc000401d000028240004220a80085824c0014
:102acc004200a9004220ae004200a8000482d300bc
:102adc00a70180000503780004027800a601880095
:102aec00004a7800a7018800144620009e0042008e
:102afc00610ab800848fd2008582d200040278006b
:102b0c0004f0a10003c02500739f9800060020006c
:102b1c0006a79800970180007e9c90008ea49000e0
:102b2c000801d0008401d000030241004220a8001b
:102b3c0085824c004200a9004220ae004200a80051
:102b4c000482d30005037800960188000402780003
:102b5c0014427800970188000440e800610ab8002c
:102b6c00848fd2008582d2000402780004f0a10088
:102b7c0006c0250016a798000700200027a798007c
:102b8c001ea49000aea490008800d0000401d000d8
:102b9c00028240004220a80085824c004200a9001d
:102bac004220ae004200a8000482d300a70180009e
:102bbc000503780004027800a6018800004a78001a
:102bcc00a7018800244620009e004200610ab8003c
:102bdc00848fd2008582d2000402780004f0a10018
:102bec0003c0250033a798000600200046a79800d4
:102bfc00970180003ea49000cea490000801d00064
:102c0c008401d000030241004220a80085824c00c0
:102c1c004200a9004220ae004200a8000482d3006a
:102c2c0005037800960188000402780014427800ad
:102c3c00970188000440e800610ab800848fd20034
:102c4c008582d2000402780004f0a10006c02500a1
:102c5c0056a798000700200067a798005ea4900074
:102c6c00eea490008800d0000401d0000282400045
:102c7c004220a80085824c004200a9004220ae00f0
:102c8c004200a8000482d300a7018000050378004d
:102c9c0004027800a6018800004a7800a701880089
:102cac00344620009e004200610ab800848fd20096
:102cbc008582d2000402780004f0a10003c0250034
:102ccc0073a798000600200006af980097018000bb
:102cdc007ea490008eac90000801d0008401d0003e
:102cec00030241004220a80085824c004200a9004a
:102cfc004220ae004200a8000482d30005037800f5
:102d0c00960188000402780014427800970188002c
:102d1c000440e800610ab800848fd2008582d2009a
:102d2c000402780004f0a10006c0250016af98003c
:102d3c000700200027af98001eac9000aeac9000ae
:102d4c008800d0000401d000028240004220a8007c
:102d5c0085824c004200a9004220ae004200a8002f
:102d6c000482d300a70180000503780004027800d8
:102d7c00a6018800004a7800a7018800444620007c
:102d8c009e004200610ab800848fd2008582d20076
:102d9c000402780004f0a10003c0250033af9800b2
:102dac000600200046af9800970180003eac9000d2
:102dbc00ceac90000801d0008401d0000302410089
:102dcc004220a80085824c004200a9004220ae009f
:102ddc004200a8000482d300050378009601880005
:102dec000402780014427800970188000440e8003f
:102dfc00610ab800848fd2008582d2000402780068
:102e0c0004f0a10006c0250056af98000700200072
:102e1c0067af98005eac9000eeac90008800d000dc
:102e2c000401d000028240004220a80085824c00a0
:102e3c004200a9004220ae004200a8000482d30048
:102e4c00a70180000503780004027800a601880021
:102e5c00004a7800a7018800544620009e004200da
:102e6c00610ab800848fd2008582d20004027800f7
:102e7c0004f0a10003c0250073af980006002000e9
:102e8c0006b79800970180007eac90008eb490003d
:102e9c000801d0008401d000030241004220a800a8
:102eac0085824c004200a9004220ae004200a800de
:102ebc000482d30005037800960188000402780090
:102ecc0014427800970188000440e800610ab800b9
:102edc00848fd2008582d2000402780004f0a10015
:102eec0006c0250016b798000700200027b79800e9
:102efc001eb49000aeb490008800d0000401d00045
:102f0c00028240004220a80085824c004200a900a9
:102f1c004220ae004200a8000482d300a70180002a
:102f2c000503780004027800a6018800004a7800a6
:102f3c00a7018800644620009e004200610ab80088
:102f4c00848fd2008582d2000402780004f0a100a4
:102f5c0003c0250033b798000600200046b7980040
:102f6c00970180003eb49000ceb490000801d000d0
:102f7c008401d000030241004220a80085824c004d
:102f8c004200a9004220ae004200a8000482d300f7
:102f9c00050378009601880004027800144278003a
:102fac00970188000440e800610ab800848fd200c1
:102fbc008582d2000402780004f0a10006c025002e
:102fcc0056b798000700200067b798005eb49000d1
:102fdc00eeb490008800d0000401d00002824000c2
:102fec004220a80085824c004200a9004220ae007d
:102ffc004200a8000482d300a701800005037800da
:10300c0004027800a6018800004a7800a701880015
:10301c00145020009e004200610ab800848fd20038
:10302c008582d2000402780004f0a10003c02500c0
:10303c0073b798000600200006bf98009701800027
:10304c007eb490008ebc90000801d0008401d000aa
:10305c00030241004220a80085824c004200a900d6
:10306c004220ae004200a8000482d3000503780081
:10307c0096018800040278001442780097018800b9
:10308c000440e800610ab800848fd2008582d20027
:10309c000402780004f0a10006c0250016bf9800b9
:1030ac000700200027bf98001ebc9000aebc90000b
:1030bc008800d0000401d000028240004220a80009
:1030cc0085824c004200a9004220ae004200a800bc
:1030dc000482d300a7018000050378000402780065
:1030ec00a6018800004a7800a7018800245020001f
:1030fc009e004200610ab800848fd2008582d20003
:10310c000402780004f0a10003c0250033bf98002e
:10311c000600200046bf9800970180003ebc90003e
:10312c00cebc90000801d0008401d0000302410005
:10313c004220a80085824c004200a9004220ae002b
:10314c004200a8000482d300050378009601880091
:10315c000402780014427800970188000440e800cb
:10316c00610ab800848fd2008582d20004027800f4
:10317c0004f0a10006c0250056bf980007002000ef
:10318c0067bf98005ebc9000eebc90008800d00039
:10319c000401d000028240004220a80085824c002d
:1031ac004200a9004220ae004200a8000482d300d5
:1031bc00a70180000503780004027800a6018800ae
:1031cc00004a7800a7018800345020009e0042007d
:1031dc00610ab800848fd2008582d2000402780084
:1031ec0004f0a10003c0250073bf98000600200066
:1031fc0006079900970180007ebc90008e04910018
:10320c000801d0008401d000030241004220a80034
:10321c0085824c004200a9004220ae004200a8006a
:10322c000482d3000503780096018800040278001c
:10323c0014427800970188000440e800610ab80045
:10324c00848fd2008582d2000402780004f0a100a1
:10325c0006c02500160799000700200027079900d3
:10326c001e049100ae0491008800d0000401d0002f
:10327c00028240004220a80085824c004200a90036
:10328c004220ae004200a8000482d300a7018000b7
:10329c000503780004027800a6018800004a780033
:1032ac00a7018800445020009e004200610ab8002b
:1032bc00848fd2008582d2000402780004f0a10031
:1032cc0003c025003307990006002000460799002b
:1032dc00970180003e049100ce0491000801d000bb
:1032ec008401d000030241004220a80085824c00da
:1032fc004200a9004220ae004200a8000482d30084
:10330c0005037800960188000402780014427800c6
:10331c00970188000440e800610ab800848fd2004d
:10332c008582d2000402780004f0a10006c02500ba
:10333c005607990007002000670799005e0491006a
:10334c00ee0491008800d0000401d00002824000fd
:10335c004220a80085824c004200a9004220ae0009
:10336c004200a8000482d300a70180000503780066
:10337c0004027800a6018800004a7800a7018800a2
:10338c00545020009e004200610ab800848fd20085
:10339c008582d2000402780004f0a10003c025004d
:1033ac007307990006002000060f99009701800012
:1033bc007e0491008e0c91000801d0008401d00095
:1033cc00030241004220a80085824c004200a90063
:1033dc004220ae004200a8000482d300050378000e
:1033ec009601880004027800144278009701880046
:1033fc000440e800610ab800848fd2008582d200b4
:10340c000402780004f0a10006c02500160f9900f4
:10341c0007002000270f99001e0c9100ae0c9100a4
:10342c008800d0000401d000028240004220a80095
:10343c0085824c004200a9004220ae004200a80048
:10344c000482d300a70180000503780004027800f1
:10345c00a6018800004a7800a7018800645020006b
:10346c009e004200610ab800848fd2008582d2008f
:10347c000402780004f0a10003c02500330f99006a
:10348c0006002000460f9900970180003e0c910029
:10349c00ce0c91000801d0008401d0000302410041
:1034ac004220a80085824c004200a9004220ae00b8
:1034bc004200a8000482d30005037800960188001e
:1034cc000402780014427800970188000440e80058
:1034dc00610ab800848fd2008582d2000402780081
:1034ec0004f0a10006c02500560f9900070020002b
:1034fc00670f99005e0c9100ee0c91008800d000d3
:10350c000401d000028240004220a80085824c00b9
:10351c004200a9004220ae004200a8000482d30061
:10352c00a70180000503780004027800a60188003a
:10353c00004a7800a7018800145a20009e0042001f
:10354c00610ab800848fd2008582d2000402780010
:10355c0004f0a10003c02500730f990006002000a1
:10356c0006179900970180007e0c91008e14910033
:10357c000801d0008401d000030241004220a800c1
:10358c0085824c004200a9004220ae004200a800f7
:10359c000482d300050378009601880004027800a9
:1035ac0014427800970188000440e800610ab800d2
:1035bc00848fd2008582d2000402780004f0a1002e
:1035cc0006c0250016179900070020002717990040
:1035dc001e149100ae1491008800d0000401d0009c
:1035ec00028240004220a80085824c004200a900c3
:1035fc004220ae004200a8000482d300a701800044
:10360c000503780004027800a6018800004a7800bf
:10361c00a7018800245a20009e004200610ab800cd
:10362c00848fd2008582d2000402780004f0a100bd
:10363c0003c0250033179900060020004617990097
:10364c00970180003e149100ce1491000801d00027
:10365c008401d000030241004220a80085824c0066
:10366c004200a9004220ae004200a8000482d30010
:10367c000503780096018800040278001442780053
:10368c00970188000440e800610ab800848fd200da
:10369c008582d2000402780004f0a10006c0250047
:1036ac005617990007002000671799005e149100c7
:1036bc00ee1491008800d0000401d000028240007a
:1036cc004220a80085824c004200a9004220ae0096
:1036dc004200a8000482d300a701800005037800f3
:1036ec0004027800a6018800004a7800a70188002f
:1036fc00345a20009e004200610ab800848fd20028
:10370c008582d2000402780004f0a10003c02500d9
:10371c007317990006002000061f9900970180007e
:10372c007e1491008e1c91000801d0008401d00001
:10373c00030241004220a80085824c004200a900ef
:10374c004220ae004200a8000482d300050378009a
:10375c0096018800040278001442780097018800d2
:10376c000440e800610ab800848fd2008582d20040
:10377c000402780004f0a10006c02500161f990071
:10378c0007002000271f99001e1c9100ae1c910001
:10379c008800d0000401d000028240004220a80022
:1037ac0085824c004200a9004220ae004200a800d5
:1037bc000482d300a701800005037800040278007e
:1037cc00a6018800004a7800a7018800445a20000e
:1037dc009e004200610ab800848fd2008582d2001c
:1037ec000402780004f0a10003c02500331f9900e7
:1037fc0006002000461f9900970180003e1c910096
:10380c00ce1c91000801d0008401d00003024100bd
:10381c004220a80085824c004200a9004220ae0044
:10382c004200a8000482d3000503780096018800aa
:10383c000402780014427800970188000440e800e4
:10384c00610ab800848fd2008582d200040278000d
:10385c0004f0a10006c02500561f990007002000a7
:10386c00671f99005e1c9100ee1c91008800d0002f
:10387c000401d000028240004220a80085824c0046
:10388c004200a9004220ae004200a8000482d300ee
:10389c00a70180000503780004027800a6018800c7
:1038ac00004a7800a7018800545a20009e0042006c
:1038bc00610ab800848fd2008582d200040278009d
:1038cc0004f0a10003c02500731f9900060020001e
:1038dc0006279900970180007e1c91008e24910090
:1038ec000801d0008401d000030241004220a8004e
:1038fc0085824c004200a9004220ae004200a80084
:10390c000482d30005037800960188000402780035
:10391c0014427800970188000440e800610ab8005e
:10392c00848fd2008582d2000402780004f0a100ba
:10393c0006c02500162799000700200027279900ac
:10394c001e249100ae2491008800d0000401d00008
:10395c00028240004220a80085824c004200a9004f
:10396c004220ae004200a8000482d300a7018000d0
:10397c000503780004027800a6018800004a78004c
:10398c00a7018800645a20009e004200610ab8001a
:10399c00848fd2008582d2000402780004f0a1004a
:1039ac0003c0250033279900060020004627990004
:1039bc00970180003e249100ce2491000801d00094
:1039cc008401d000030241004220a80085824c00f3
:1039dc004200a9004220ae004200a8000482d3009d
:1039ec0005037800960188000402780014427800e0
:1039fc00970188000440e800610ab800848fd20067
:103a0c008582d2000402780004f0a10006c02500d3
:103a1c005627990007002000672799005e24910023
:103a2c00ee2491008800d0000401d00002824000f6
:103a3c004220a80085824c004200a9004220ae0022
:103a4c004200a8000482d300a7018000050378007f
:103a5c0004027800a6018800004a7800a7018800bb
:103a6c00046420009e004200610ab800848fd200da
:103a7c008582d2000402780004f0a10003c0250066
:103a8c007327990006002000062f990097018000eb
:103a9c007e2491008e2c91000801d0008401d0006e
:103aac00030241004220a80085824c004200a9007c
:103abc004220ae004200a8000482d3000503780027
:103acc00960188000402780014427800970188005f
:103adc000440e800610ab800848fd2008582d200cd
:103aec000402780004f0a10006c02500162f9900ee
:103afc0007002000272f99001e2c9100ae2c91005e
:103b0c008800d0000401d000028240004220a800ae
:103b1c0085824c004200a9004220ae004200a80061
:103b2c000482d300a701800005037800040278000a
:103b3c00a6018800004a7800a701880014642000c0
:103b4c009e004200610ab800848fd2008582d200a8
:103b5c000402780004f0a10003c02500332f990063
:103b6c0006002000462f9900970180003e2c910002
:103b7c00ce2c91000801d0008401d000030241003a
:103b8c004220a80085824c004200a9004220ae00d1
:103b9c004200a8000482d300050378009601880037
:103bac000402780014427800970188000440e80071
:103bbc00610ab800848fd2008582d200040278009a
:103bcc0004f0a10006c02500562f99000700200024
:103bdc00672f99005e2c9100ee2c91008800d0008c
:103bec000401d000028240004220a80085824c00d3
:103bfc004200a9004220ae004200a8000482d3007b
:103c0c00a70180000503780004027800a601880053
:103c1c00004a7800a7018800246420009e0042001e
:103c2c00610ab800848fd2008582d2000402780029
:103c3c0004f0a10003c02500732f9900060020009a
:103c4c0006379900970180007e2c91008e349100ec
:103c5c000801d0008401d000030241004220a800da
:103c6c0085824c004200a9004220ae004200a80010
:103c7c000482d300050378009601880004027800c2
:103c8c0014427800970188000440e800610ab800eb
:103c9c00848fd2008582d2000402780004f0a10047
:103cac0006c0250016379900070020002737990019
:103cbc001e349100ae3491008800d0000401d00075
:103ccc00028240004220a80085824c004200a900dc
:103cdc004220ae004200a8000482d300a70180005d
:103cec000503780004027800a6018800004a7800d9
:103cfc00a7018800346420009e004200610ab800cd
:103d0c00848fd2008582d2000402780004f0a100d6
:103d1c0003c0250033379900060020004637990070
:103d2c00970180003e349100ce3491000801d00000
:103d3c008401d000030241004220a80085824c007f
:103d4c004200a9004220ae004200a8000482d30029
:103d5c00050378009601880004027800144278006c
:103d6c00970188000440e800610ab800848fd200f3
:103d7c008582d2000402780004f0a10006c0250060
:103d8c005637990007002000673799005e34910080
:103d9c00ee3491008800d0000401d0000282400073
:103dac004220a80085824c004200a9004220ae00af
:103dbc004200a8000482d300a7018000050378000c
:103dcc0004027800a6018800004a7800a701880048
:103ddc00446420009e004200610ab800848fd20027
:103dec008582d2000402780004f0a10003c02500f3
:103dfc007337990006002000063f99009701800058
:103e0c007e3491008e3c91000801d0008401d000da
:103e1c00030241004220a80085824c004200a90008
:103e2c004220ae004200a8000482d30005037800b3
:103e3c0096018800040278001442780097018800eb
:103e4c000440e800610ab800848fd2008582d20059
:103e5c000402780004f0a10006c02500163f99006a
:103e6c0007002000273f99001e3c9100ae3c9100ba
:103e7c008800d0000401d000028240004220a8003b
:103e8c0085824c004200a9004220ae004200a800ee
:103e9c000482d300a7018000050378000402780097
:103eac00a6018800004a7800a7018800546420000d
:103ebc009e004200610ab800848fd2008582d20035
:103ecc000402780004f0a10003c02500333f9900e0
:103edc0006002000463f9900970180003e3c91006f
:103eec00ce3c91000801d0008401d00003024100b7
:103efc004220a80085824c004200a9004220ae005e
:103f0c004200a8000482d3000503780096018800c3
:103f1c000402780014427800970188000440e800fd
:103f2c00610ab800848fd2008582d2000402780026
:103f3c0004f0a10006c02500563f990007002000a0
:103f4c00673f99005e3c9100ee3c91008800d000e8
:103f5c000401d000028240004220a80085824c005f
:103f6c004200a9004220ae004200a8000482d30007
:103f7c00a70180000503780004027800a6018800e0
:103f8c00004a7800a7018800646420009e0042006b
:103f9c00610ab800848fd2008582d20004027800b6
:103fac0004f0a10003c02500733f99000600200017
:103fbc0006879900970180007e3c91008e849100c9
:103fcc000801d0008401d000030241004220a80067
:103fdc0085824c004200a9004220ae004200a8009d
:103fec000482d3000503780096018800040278004f
:103ffc0014427800970188000440e800610ab80078
:10400c00848fd2008582d2000402780004f0a100d3
:10401c0006c0250016879900070020002787990005
:10402c001e849100ae8491008800d0000401d00061
:10403c00028240004220a80085824c004200a90068
:10404c004220ae004200a8000482d300a7018000e9
:10405c000503780004027800a6018800004a780065
:10406c00a7018800746420009e004200610ab80019
:10407c00848fd2008582d2000402780004f0a10063
:10408c0003c025003387990006002000468799005d
:10409c00970180003e849100ce8491000801d000ed
:1040ac008401d000030241004220a80085824c000c
:1040bc004200a9004220ae004200a8000482d300b6
:1040cc0005037800960188000402780014427800f9
:1040dc00970188000440e800610ab800848fd20080
:1040ec008582d2000402780004f0a10006c02500ed
:1040fc005687990007002000678799005e8491001d
:10410c00ee8491008800d0000401d00002824000af
:10411c004220a80085824c004200a9004220ae003b
:10412c004200a8000482d300a70180000503780098
:10413c0004027800a6018800004a7800a7018800d4
:10414c00046e20009e004200610ab800848fd200e9
:10415c008582d2000402780004f0a10003c025007f
:10416c007387990006002000068f99009701800044
:10417c007e8491008e8c91000801d0008401d000c7
:10418c00030241004220a80085824c004200a90095
:10419c004220ae004200a8000482d3000503780040
:1041ac009601880004027800144278009701880078
:1041bc000440e800610ab800848fd2008582d200e6
:1041cc000402780004f0a10006c02500168f9900a7
:1041dc0007002000278f99001e8c9100ae8c910057
:1041ec008800d0000401d000028240004220a800c8
:1041fc0085824c004200a9004220ae004200a8007b
:10420c000482d300a7018000050378000402780023
:10421c00a6018800004a7800a7018800146e2000cf
:10422c009e004200610ab800848fd2008582d200c1
:10423c000402780004f0a10003c02500338f99001c
:10424c0006002000468f9900970180003e8c91005b
:10425c00ce8c91000801d0008401d00003024100f3
:10426c004220a80085824c004200a9004220ae00ea
:10427c004200a8000482d300050378009601880050
:10428c000402780014427800970188000440e8008a
:10429c00610ab800848fd2008582d20004027800b3
:1042ac0004f0a10006c02500568f990007002000dd
:1042bc00678f99005e8c9100ee8c91008800d00085
:1042cc000401d000028240004220a80085824c00ec
:1042dc004200a9004220ae004200a8000482d30094
:1042ec00a70180000503780004027800a60188006d
:1042fc00004a7800a7018800246e20009e0042002e
:10430c00610ab800848fd2008582d2000402780042
:10431c0004f0a10003c02500738f99000600200053
:10432c0006979900970180007e8c91008e949100e5
:10433c000801d0008401d000030241004220a800f3
:10434c0085824c004200a9004220ae004200a80029
:10435c000482d300050378009601880004027800db
:10436c0014427800970188000440e800610ab80004
:10437c00848fd2008582d2000402780004f0a10060
:10438c0006c0250016979900070020002797990072
:10439c001e949100ae9491008800d0000401d000ce
:1043ac00028240004220a80085824c004200a900f5
:1043bc004220ae004200a8000482d300a701800076
:1043cc000503780004027800a6018800004a7800f2
:1043dc00a7018800346e20009e004200610ab800dc
:1043ec00848fd2008582d2000402780004f0a100f0
:1043fc0003c02500339799000600200046979900ca
:10440c00970180003e949100ce9491000801d00059
:10441c008401d000030241004220a80085824c0098
:10442c004200a9004220ae004200a8000482d30042
:10443c000503780096018800040278001442780085
:10444c00970188000440e800610ab800848fd2000c
:10445c008582d2000402780004f0a10006c0250079
:10446c005697990007002000679799005e94910079
:10447c00ee9491008800d0000401d000028240002c
:10448c004220a80085824c004200a9004220ae00c8
:10449c004200a8000482d300a70180000503780025
:1044ac0004027800a6018800004a7800a701880061
:1044bc00446e20009e004200610ab800848fd20036
:1044cc008582d2000402780004f0a10003c025000c
:1044dc007397990006002000069f990097018000b1
:1044ec007e9491008e9c91000801d0008401d00034
:1044fc00030241004220a80085824c004200a90022
:10450c004220ae004200a8000482d30005037800cc
:10451c009601880004027800144278009701880004
:10452c000440e800610ab800848fd2008582d20072
:10453c000402780004f0a10006c02500169f990023
:10454c0007002000279f99001e9c9100ae9c9100b3
:10455c008800d0000401d000028240004220a80054
:10456c0085824c004200a9004220ae004200a80007
:10457c000482d300a70180000503780004027800b0
:10458c00a6018800004a7800a7018800546e20001c
:10459c009e004200610ab800848fd2008582d2004e
:1045ac000402780004f0a10003c02500339f990099
:1045bc0006002000469f9900970180003e9c9100c8
:1045cc00ce9c91000801d0008401d0000302410070
:1045dc004220a80085824c004200a9004220ae0077
:1045ec004200a8000482d3000503780096018800dd
:1045fc000402780014427800970188000440e80017
:10460c00610ab800848fd2008582d200040278003f
:10461c0004f0a10006c02500569f99000700200059
:10462c00679f99005e9c9100ee9c91008800d000e1
:10463c000401d000028240004220a80085824c0078
:10464c004200a9004220ae004200a8000482d30020
:10465c00a70180000503780004027800a6018800f9
:10466c00004a7800a7018800646e20009e0042007a
:10467c00610ab800848fd2008582d20004027800cf
:10468c0004f0a10003c02500739f990006002000d0
:10469c0006a79900970180007e9c91008ea4910042
:1046ac000801d0008401d000030241004220a80080
:1046bc0085824c004200a9004220ae004200a800b6
:1046cc000482d30005037800960188000402780068
:1046dc0014427800970188000440e800610ab80091
:1046ec00848fd2008582d2000402780004f0a100ed
:1046fc0006c0250016a799000700200027a79900df
:10470c001ea49100aea491008800d0000401d0003a
:10471c00028240004220a80085824c004200a90081
:10472c004220ae004200a8000482d300a701800002
:10473c000503780004027800a6018800004a78007e
:10474c00a7018800746e20009e004200610ab80028
:10475c00848fd2008582d2000402780004f0a1007c
:10476c0003c0250033a799000600200046a7990036
:10477c00970180003ea49100cea491000801d000c6
:10478c008401d000030241004220a80085824c0025
:10479c004200a9004220ae004200a8000482d300cf
:1047ac000503780096018800040278001442780012
:1047bc00970188000440e800610ab800848fd20099
:1047cc008582d2000402780004f0a10006c0250006
:1047dc0056a799000700200067a799005ea49100d6
:1047ec00eea491008800d0000401d00002824000a9
:1047fc004220a80085824c004200a9004220ae0055
:10480c004200a8000482d300a701800005037800b1
:10481c0004027800a6018800004a7800a7018800ed
:10482c00047820009e004200610ab800848fd200f8
:10483c008582d2000402780004f0a10003c0250098
:10484c0073a799000600200006af9900970180001d
:10485c007ea491008eac91000801d0008401d000a0
:10486c00030241004220a80085824c004200a900ae
:10487c004220ae004200a8000482d3000503780059
:10488c009601880004027800144278009701880091
:10489c000440e800610ab800848fd2008582d200ff
:1048ac000402780004f0a10006c0250016af9900a0
:1048bc000700200027af99001eac9100aeac910010
:1048cc008800d0000401d000028240004220a800e1
:1048dc0085824c004200a9004220ae004200a80094
:1048ec000482d300a701800005037800040278003d
:1048fc00a6018800004a7800a701880014782000df
:10490c009e004200610ab800848fd2008582d200da
:10491c000402780004f0a10003c0250033af990015
:10492c000600200046af9900970180003eac910034
:10493c00ceac91000801d0008401d00003024100ec
:10494c004220a80085824c004200a9004220ae0003
:10495c004200a8000482d300050378009601880069
:10496c000402780014427800970188000440e800a3
:10497c00610ab800848fd2008582d20004027800cc
:10498c0004f0a10006c0250056af990007002000d6
:10499c0067af99005eac9100eeac91008800d0003e
:1049ac000401d000028240004220a80085824c0005
:1049bc004200a9004220ae004200a8000482d300ad
:1049cc00a70180000503780004027800a601880086
:1049dc00004a7800a7018800247820009e0042003d
:1049ec00610ab800848fd2008582d200040278005c
:1049fc0004f0a10003c0250073af9900060020004d
:104a0c0006b79900970180007eac91008eb491009e
:104a1c000801d0008401d000030241004220a8000c
:104a2c0085824c004200a9004220ae004200a80042
:104a3c000482d300050378009601880004027800f4
:104a4c0014427800970188000440e800610ab8001d
:104a5c00848fd2008582d2000402780004f0a10079
:104a6c0006c0250016b799000700200027b799004b
:104a7c001eb49100aeb491008800d0000401d000a7
:104a8c00028240004220a80085824c004200a9000e
:104a9c004220ae004200a8000482d300a70180008f
:104aac000503780004027800a6018800004a78000b
:104abc00a7018800347820009e004200610ab800eb
:104acc00848fd2008582d2000402780004f0a10009
:104adc0003c0250033b799000600200046b79900a3
:104aec00970180003eb49100ceb491000801d00033
:104afc008401d000030241004220a80085824c00b2
:104b0c004200a9004220ae004200a8000482d3005b
:104b1c00050378009601880004027800144278009e
:104b2c00970188000440e800610ab800848fd20025
:104b3c008582d2000402780004f0a10006c0250092
:104b4c0056b799000700200067b799005eb4910032
:104b5c00eeb491008800d0000401d0000282400025
:104b6c004220a80085824c004200a9004220ae00e1
:104b7c004200a8000482d300a7018000050378003e
:104b8c0004027800a6018800004a7800a70188007a
:104b9c00447820009e004200610ab800848fd20045
:104bac008582d2000402780004f0a10003c0250025
:104bbc0073b799000600200006bf9900970180008a
:104bcc007eb491008ebc91000801d0008401d0000d
:104bdc00030241004220a80085824c004200a9003b
:104bec004220ae004200a8000482d30005037800e6
:104bfc00960188000402780014427800970188001e
:104c0c000440e800610ab800848fd2008582d2008b
:104c1c000402780004f0a10006c0250016bf99001c
:104c2c000700200027bf99001ebc9100aebc91006c
:104c3c008800d0000401d000028240004220a8006d
:104c4c0085824c004200a9004220ae004200a80020
:104c5c000482d300a70180000503780004027800c9
:104c6c00a6018800004a7800a7018800547820002b
:104c7c009e004200610ab800848fd2008582d20067
:104c8c000402780004f0a10003c0250033bf990092
:104c9c000600200046bf9900970180003ebc9100a1
:104cac00cebc91000801d0008401d0000302410069
:104cbc004220a80085824c004200a9004220ae0090
:104ccc004200a8000482d3000503780096018800f6
:104cdc000402780014427800970188000440e80030
:104cec00610ab800848fd2008582d2000402780059
:104cfc0004f0a10006c0250056bf99000700200053
:104d0c0067bf99005ebc9100eebc91008800d0009a
:104d1c000401d000028240004220a80085824c0091
:104d2c004200a9004220ae004200a8000482d30039
:104d3c00a70180000503780004027800a601880012
:104d4c00004a7800a7018800647820009e00420089
:104d5c00610ab800848fd2008582d20004027800e8
:104d6c0004f0a10003c0250073bf990006002000c9
:104d7c0006079a00970180007ebc91008e04920079
:104d8c000801d0008401d000030241004220a80099
:104d9c0085824c004200a9004220ae004200a800cf
:104dac000482d30005037800960188000402780081
:104dbc0014427800970188000440e800610ab800aa
:104dcc00848fd2008582d2000402780004f0a10006
:104ddc0006c0250016079a000700200027079a0036
:104dec001e049200ae0492008800d0000401d00092
:104dfc00028240004220a80085824c004200a9009b
:104e0c004220ae004200a8000482d300a70180001b
:104e1c000503780004027800a6018800004a780097
:104e2c00a7018800747820009e004200610ab80037
:104e3c00848fd2008582d2000402780004f0a10095
:104e4c0003c0250033079a000600200046079a008d
:104e5c00970180003e049200ce0492000801d0001d
:104e6c008401d000030241004220a80085824c003e
:104e7c004200a9004220ae004200a8000482d300e8
:104e8c00050378009601880004027800144278002b
:104e9c00970188000440e800610ab800848fd200b2
:104eac008582d2000402780004f0a10006c025001f
:104ebc0056079a000700200067079a005e049200cc
:104ecc00ee0492008800d0000401d0000282400061
:104edc004220a80085824c004200a9004220ae006e
:104eec004200a8000482d300a701800005037800cb
:104efc0004027800a6018800004a7800a701880007
:104f0c00048220009e004200610ab800848fd20007
:104f1c008582d2000402780004f0a10003c02500b1
:104f2c0073079a0006002000060f9a009701800074
:104f3c007e0492008e0c92000801d0008401d000f7
:104f4c00030241004220a80085824c004200a900c7
:104f5c004220ae004200a8000482d3000503780072
:104f6c0096018800040278001442780097018800aa
:104f7c000440e800610ab800848fd2008582d20018
:104f8c000402780004f0a10006c02500160f9a0058
:104f9c0007002000270f9a001e0c9200ae0c920006
:104fac008800d0000401d000028240004220a800fa
:104fbc0085824c004200a9004220ae004200a800ad
:104fcc000482d300a7018000050378000402780056
:104fdc00a6018800004a7800a701880014822000ee
:104fec009e004200610ab800848fd2008582d200f4
:104ffc000402780004f0a10003c02500330f9a00ce
:10500c0006002000460f9a00970180003e0c92008b
:10501c00ce0c92000801d0008401d00003024100a4
:10502c004220a80085824c004200a9004220ae001c
:10503c004200a8000482d300050378009601880082
:10504c000402780014427800970188000440e800bc
:10505c00610ab800848fd2008582d20004027800e5
:10506c0004f0a10006c02500560f9a00070020008e
:10507c00670f9a005e0c9200ee0c92008800d00034
:10508c000401d000028240004220a80085824c001e
:10509c004200a9004220ae004200a8000482d300c6
:1050ac00a70180000503780004027800a60188009f
:1050bc00004a7800a7018800248220009e0042004c
:1050cc00610ab800848fd2008582d2000402780075
:1050dc0004f0a10003c02500730f9a000600200005
:1050ec0006179a00970180007e0c92008e14920095
:1050fc000801d0008401d000030241004220a80026
:10510c0085824c004200a9004220ae004200a8005b
:10511c000482d3000503780096018800040278000d
:10512c0014427800970188000440e800610ab80036
:10513c00848fd2008582d2000402780004f0a10092
:10514c0006c0250016179a000700200027179a00a2
:10515c001e149200ae1492008800d0000401d000fe
:10516c00028240004220a80085824c004200a90027
:10517c004220ae004200a8000482d300a7018000a8
:10518c000503780004027800a6018800004a780024
:10519c00a7018800348220009e004200610ab800fa
:1051ac00848fd2008582d2000402780004f0a10022
:1051bc0003c0250033179a000600200046179a00fa
:1051cc00970180003e149200ce1492000801d0008a
:1051dc008401d000030241004220a80085824c00cb
:1051ec004200a9004220ae004200a8000482d30075
:1051fc0005037800960188000402780014427800b8
:10520c00970188000440e800610ab800848fd2003e
:10521c008582d2000402780004f0a10006c02500ab
:10522c0056179a000700200067179a005e14920028
:10523c00ee1492008800d0000401d00002824000dd
:10524c004220a80085824c004200a9004220ae00fa
:10525c004200a8000482d300a70180000503780057
:10526c0004027800a6018800004a7800a701880093
:10527c00448220009e004200610ab800848fd20054
:10528c008582d2000402780004f0a10003c025003e
:10529c0073179a0006002000061f9a0097018000e1
:1052ac007e1492008e1c92000801d0008401d00064
:1052bc00030241004220a80085824c004200a90054
:1052cc004220ae004200a8000482d30005037800ff
:1052dc009601880004027800144278009701880037
:1052ec000440e800610ab800848fd2008582d200a5
:1052fc000402780004f0a10006c02500161f9a00d5
:10530c0007002000271f9a001e1c9200ae1c920062
:10531c008800d0000401d000028240004220a80086
:10532c0085824c004200a9004220ae004200a80039
:10533c000482d300a70180000503780004027800e2
:10534c00a6018800004a7800a7018800548220003a
:10535c009e004200610ab800848fd2008582d20080
:10536c000402780004f0a10003c02500331f9a004a
:10537c0006002000461f9a00970180003e1c9200f8
:10538c00ce1c92000801d0008401d0000302410021
:10539c004220a80085824c004200a9004220ae00a9
:1053ac004200a8000482d30005037800960188000f
:1053bc000402780014427800970188000440e80049
:1053cc00610ab800848fd2008582d2000402780072
:1053dc0004f0a10006c02500561f9a00070020000b
:1053ec00671f9a005e1c9200ee1c92008800d00091
:1053fc000401d000028240004220a80085824c00ab
:10540c004200a9004220ae004200a8000482d30052
:10541c00a70180000503780004027800a60188002b
:10542c00004a7800a7018800648220009e00420098
:10543c00610ab800848fd2008582d2000402780001
:10544c0004f0a10003c02500731f9a000600200081
:10545c0006279a00970180007e1c92008e249200f1
:10546c000801d0008401d000030241004220a800b2
:10547c0085824c004200a9004220ae004200a800e8
:10548c000482d3000503780096018800040278009a
:10549c0014427800970188000440e800610ab800c3
:1054ac00848fd2008582d2000402780004f0a1001f
:1054bc0006c0250016279a000700200027279a000f
:1054cc001e249200ae2492008800d0000401d0006b
:1054dc00028240004220a80085824c004200a900b4
:1054ec004220ae004200a8000482d300a701800035
:1054fc000503780004027800a6018800004a7800b1
:10550c00a7018800748220009e004200610ab80046
:10551c00848fd2008582d2000402780004f0a100ae
:10552c0003c0250033279a000600200046279a0066
:10553c00970180003e249200ce2492000801d000f6
:10554c008401d000030241004220a80085824c0057
:10555c004200a9004220ae004200a8000482d30001
:10556c000503780096018800040278001442780044
:10557c00970188000440e800610ab800848fd200cb
:10558c008582d2000402780004f0a10006c0250038
:10559c0056279a000700200067279a005e24920085
:1055ac00ee2492008800d0000401d000028240005a
:1055bc004220a80085824c004200a9004220ae0087
:1055cc004200a8000482d300a701800005037800e4
:1055dc0004027800a6018800004a7800a701880020
:1055ec00048c20009e004200610ab800848fd20017
:1055fc008582d2000402780004f0a10003c02500cb
:10560c0073279a0006002000062f9a00970180004d
:10561c007e2492008e2c92000801d0008401d000d0
:10562c00030241004220a80085824c004200a900e0
:10563c004220ae004200a8000482d300050378008b
:10564c0096018800040278001442780097018800c3
:10565c000440e800610ab800848fd2008582d20031
:10566c000402780004f0a10006c02500162f9a0051
:10567c0007002000272f9a001e2c9200ae2c9200bf
:10568c008800d0000401d000028240004220a80013
:10569c0085824c004200a9004220ae004200a800c6
:1056ac000482d300a701800005037800040278006f
:1056bc00a6018800004a7800a7018800148c2000fd
:1056cc009e004200610ab800848fd2008582d2000d
:1056dc000402780004f0a10003c02500332f9a00c7
:1056ec0006002000462f9a00970180003e2c920065
:1056fc00ce2c92000801d0008401d000030241009e
:10570c004220a80085824c004200a9004220ae0035
:10571c004200a8000482d30005037800960188009b
:10572c000402780014427800970188000440e800d5
:10573c00610ab800848fd2008582d20004027800fe
:10574c0004f0a10006c02500562f9a000700200087
:10575c00672f9a005e2c9200ee2c92008800d000ed
:10576c000401d000028240004220a80085824c0037
:10577c004200a9004220ae004200a8000482d300df
:10578c00a70180000503780004027800a6018800b8
:10579c00004a7800a7018800248c20009e0042005b
:1057ac00610ab800848fd2008582d200040278008e
:1057bc0004f0a10003c02500732f9a0006002000fe
:1057cc0006379a00970180007e2c92008e3492004e
:1057dc000801d0008401d000030241004220a8003f
:1057ec0085824c004200a9004220ae004200a80075
:1057fc000482d30005037800960188000402780027
:10580c0014427800970188000440e800610ab8004f
:10581c00848fd2008582d2000402780004f0a100ab
:10582c0006c0250016379a000700200027379a007b
:10583c001e349200ae3492008800d0000401d000d7
:10584c00028240004220a80085824c004200a90040
:10585c004220ae004200a8000482d300a7018000c1
:10586c000503780004027800a6018800004a78003d
:10587c00a7018800348c20009e004200610ab80009
:10588c00848fd2008582d2000402780004f0a1003b
:10589c0003c0250033379a000600200046379a00d3
:1058ac00970180003e349200ce3492000801d00063
:1058bc008401d000030241004220a80085824c00e4
:1058cc004200a9004220ae004200a8000482d3008e
:1058dc0005037800960188000402780014427800d1
:1058ec00970188000440e800610ab800848fd20058
:1058fc008582d2000402780004f0a10006c02500c5
:10590c0056379a000700200067379a005e349200e1
:10591c00ee3492008800d0000401d00002824000d6
:10592c004220a80085824c004200a9004220ae0013
:10593c004200a8000482d300a70180000503780070
:10594c0004027800a6018800004a7800a7018800ac
:10595c00448c20009e004200610ab800848fd20063
:10596c008582d2000402780004f0a10003c0250057
:10597c0073379a0006002000063f9a0097018000ba
:10598c007e3492008e3c92000801d0008401d0003d
:10599c00030241004220a80085824c004200a9006d
:1059ac004220ae004200a8000482d3000503780018
:1059bc009601880004027800144278009701880050
:1059cc000440e800610ab800848fd2008582d200be
:1059dc000402780004f0a10006c02500163f9a00ce
:1059ec0007002000273f9a001e3c9200ae3c92001c
:1059fc008800d0000401d000028240004220a800a0
:105a0c0085824c004200a9004220ae004200a80052
:105a1c000482d300a70180000503780004027800fb
:105a2c00a6018800004a7800a7018800548c200049
:105a3c009e004200610ab800848fd2008582d20099
:105a4c000402780004f0a10003c02500333f9a0043
:105a5c0006002000463f9a00970180003e3c9200d1
:105a6c00ce3c92000801d0008401d000030241001a
:105a7c004220a80085824c004200a9004220ae00c2
:105a8c004200a8000482d300050378009601880028
:105a9c000402780014427800970188000440e80062
:105aac00610ab800848fd2008582d200040278008b
:105abc0004f0a10006c02500563f9a000700200004
:105acc00673f9a005e3c9200ee3c92008800d0004a
:105adc000401d000028240004220a80085824c00c4
:105aec004200a9004220ae004200a8000482d3006c
:105afc00a70180000503780004027800a601880045
:105b0c00004a7800a7018800648c20009e004200a7
:105b1c00610ab800848fd2008582d200040278001a
:105b2c0004f0a10003c02500733f9a00060020007a
:105b3c0006879a00970180007e3c92008e8492002a
:105b4c000801d0008401d000030241004220a800cb
:105b5c0085824c004200a9004220ae004200a80001
:105b6c000482d300050378009601880004027800b3
:105b7c0014427800970188000440e800610ab800dc
:105b8c00848fd2008582d2000402780004f0a10038
:105b9c0006c0250016879a000700200027879a0068
:105bac001e849200ae8492008800d0000401d000c4
:105bbc00028240004220a80085824c004200a900cd
:105bcc004220ae004200a8000482d300a70180004e
:105bdc000503780004027800a6018800004a7800ca
:105bec00a7018800748c20009e004200610ab80056
:105bfc00848fd2008582d2000402780004f0a100c8
:105c0c0003c0250033879a000600200046879a00bf
:105c1c00970180003e849200ce8492000801d0004f
:105c2c008401d000030241004220a80085824c0070
:105c3c004200a9004220ae004200a8000482d3001a
:105c4c00050378009601880004027800144278005d
:105c5c00970188000440e800610ab800848fd200e4
:105c6c008582d2000402780004f0a10006c0250051
:105c7c0056879a000700200067879a005e8492007e
:105c8c00ee8492008800d0000401d0000282400013
:105c9c004220a80085824c004200a9004220ae00a0
:105cac004200a8000482d300a701800005037800fd
:105cbc0004027800a6018800004a7800a701880039
:105ccc00049620009e004200610ab800848fd20026
:105cdc008582d2000402780004f0a10003c02500e4
:105cec0073879a0006002000068f9a0097018000a7
:105cfc007e8492008e8c92000801d0008401d0002a
:105d0c00030241004220a80085824c004200a900f9
:105d1c004220ae004200a8000482d30005037800a4
:105d2c0096018800040278001442780097018800dc
:105d3c000440e800610ab800848fd2008582d2004a
:105d4c000402780004f0a10006c02500168f9a000a
:105d5c0007002000278f9a001e8c9200ae8c9200b8
:105d6c008800d0000401d000028240004220a8002c
:105d7c0085824c004200a9004220ae004200a800df
:105d8c000482d300a7018000050378000402780088
:105d9c00a6018800004a7800a7018800149620000c
:105dac009e004200610ab800848fd2008582d20026
:105dbc000402780004f0a10003c02500338f9a0080
:105dcc0006002000468f9a00970180003e8c9200be
:105ddc00ce8c92000801d0008401d0000302410057
:105dec004220a80085824c004200a9004220ae004f
:105dfc004200a8000482d3000503780096018800b5
:105e0c000402780014427800970188000440e800ee
:105e1c00610ab800848fd2008582d2000402780017
:105e2c0004f0a10006c02500568f9a000700200040
:105e3c00678f9a005e8c9200ee8c92008800d000e6
:105e4c000401d000028240004220a80085824c0050
:105e5c004200a9004220ae004200a8000482d300f8
:105e6c00a70180000503780004027800a6018800d1
:105e7c00004a7800a7018800249620009e0042006a
:105e8c00610ab800848fd2008582d20004027800a7
:105e9c0004f0a10003c02500738f9a0006002000b7
:105eac0006979a00970180007e8c92008e94920047
:105ebc000801d0008401d000030241004220a80058
:105ecc0085824c004200a9004220ae004200a8008e
:105edc000482d30005037800960188000402780040
:105eec0014427800970188000440e800610ab80069
:105efc00848fd2008582d2000402780004f0a100c5
:105f0c0006c0250016979a000700200027979a00d4
:105f1c001e949200ae9492008800d0000401d00030
:105f2c00028240004220a80085824c004200a90059
:105f3c004220ae004200a8000482d300a7018000da
:105f4c000503780004027800a6018800004a780056
:105f5c00a7018800349620009e004200610ab80018
:105f6c00848fd2008582d2000402780004f0a10054
:105f7c0003c0250033979a000600200046979a002c
:105f8c00970180003e949200ce9492000801d000bc
:105f9c008401d000030241004220a80085824c00fd
:105fac004200a9004220ae004200a8000482d300a7
:105fbc0005037800960188000402780014427800ea
:105fcc00970188000440e800610ab800848fd20071
:105fdc008582d2000402780004f0a10006c02500de
:105fec0056979a000700200067979a005e949200db
:105ffc00ee9492008800d0000401d0000282400090
:10600c004220a80085824c004200a9004220ae002c
:10601c004200a8000482d300a70180000503780089
:10602c0004027800a6018800004a7800a7018800c5
:10603c00449620009e004200610ab800848fd20072
:10604c008582d2000402780004f0a10003c0250070
:10605c0073979a0006002000069f9a009701800013
:10606c007e9492008e9c92000801d0008401d00096
:10607c00030241004220a80085824c004200a90086
:10608c004220ae004200a8000482d3000503780031
:10609c009601880004027800144278009701880069
:1060ac000440e800610ab800848fd2008582d200d7
:1060bc000402780004f0a10006c02500169f9a0087
:1060cc0007002000279f9a001e9c9200ae9c920015
:1060dc008800d0000401d000028240004220a800b9
:1060ec0085824c004200a9004220ae004200a8006c
:1060fc000482d300a7018000050378000402780015
:10610c00a6018800004a7800a70188005496200058
:10611c009e004200610ab800848fd2008582d200b2
:10612c000402780004f0a10003c02500339f9a00fc
:10613c0006002000469f9a00970180003e9c92002a
:10614c00ce9c92000801d0008401d00003024100d3
:10615c004220a80085824c004200a9004220ae00db
:10616c004200a8000482d300050378009601880041
:10617c000402780014427800970188000440e8007b
:10618c00610ab800848fd2008582d20004027800a4
:10619c0004f0a10006c02500569f9a0007002000bd
:1061ac00679f9a005e9c9200ee9c92008800d00043
:1061bc000401d000028240004220a80085824c00dd
:1061cc004200a9004220ae004200a8000482d30085
:1061dc00a70180000503780004027800a60188005e
:1061ec00004a7800a7018800649620009e004200b7
:1061fc00610ab800848fd2008582d2000402780034
:10620c0004f0a10003c02500739f9a000600200033
:10621c0006a79a00970180007e9c92008ea49200a3
:10622c000801d0008401d000030241004220a800e4
:10623c0085824c004200a9004220ae004200a8001a
:10624c000482d300050378009601880004027800cc
:10625c0014427800970188000440e800610ab800f5
:10626c00848fd2008582d2000402780004f0a10051
:10627c0006c0250016a79a000700200027a79a0041
:10628c001ea49200aea492008800d0000401d0009d
:10629c00028240004220a80085824c004200a900e6
:1062ac004220ae004200a8000482d300a701800067
:1062bc000503780004027800a6018800004a7800e3
:1062cc00a7018800749620009e004200610ab80065
:1062dc00848fd2008582d2000402780004f0a100e1
:1062ec0003c0250033a79a000600200046a79a0099
:1062fc00970180003ea49200cea492000801d00029
:10630c008401d000030241004220a80085824c0089
:10631c004200a9004220ae004200a8000482d30033
:10632c000503780096018800040278001442780076
:10633c00970188000440e800610ab800848fd200fd
:10634c008582d2000402780004f0a10006c025006a
:10635c0056a79a000700200067a79a005ea4920037
:10636c00eea492008800d0000401d000028240000c
:10637c004220a80085824c004200a9004220ae00b9
:10638c004200a8000482d300a70180000503780016
:10639c0004027800a6018800004a7800a701880052
:1063ac0004a020009e004200610ab800848fd20035
:1063bc008582d2000402780004f0a10003c02500fd
:1063cc0073a79a000600200006af9a009701800080
:1063dc007ea492008eac92000801d0008401d00003
:1063ec00030241004220a80085824c004200a90013
:1063fc004220ae004200a8000482d30005037800be
:10640c0096018800040278001442780097018800f5
:10641c000440e800610ab800848fd2008582d20063
:10642c000402780004f0a10006c0250016af9a0003
:10643c000700200027af9a001eac9200aeac920071
:10644c008800d0000401d000028240004220a80045
:10645c0085824c004200a9004220ae004200a800f8
:10646c000482d300a70180000503780004027800a1
:10647c00a6018800004a7800a701880014a020001b
:10648c009e004200610ab800848fd2008582d2003f
:10649c000402780004f0a10003c0250033af9a0079
:1064ac000600200046af9a00970180003eac920097
:1064bc00ceac92000801d0008401d0000302410050
:1064cc004220a80085824c004200a9004220ae0068
:1064dc004200a8000482d3000503780096018800ce
:1064ec000402780014427800970188000440e80008
:1064fc00610ab800848fd2008582d2000402780031
:10650c0004f0a10006c0250056af9a000700200039
:10651c0067af9a005eac9200eeac92008800d0009f
:10652c000401d000028240004220a80085824c0069
:10653c004200a9004220ae004200a8000482d30011
:10654c00a70180000503780004027800a6018800ea
:10655c00004a7800a701880024a020009e00420079
:10656c00610ab800848fd2008582d20004027800c0
:10657c0004f0a10003c0250073af9a0006002000b0
:10658c0006b79a00970180007eac92008eb4920000
:10659c000801d0008401d000030241004220a80071
:1065ac0085824c004200a9004220ae004200a800a7
:1065bc000482d30005037800960188000402780059
:1065cc0014427800970188000440e800610ab80082
:1065dc00848fd2008582d2000402780004f0a100de
:1065ec0006c0250016b79a000700200027b79a00ae
:1065fc001eb49200aeb492008800d0000401d0000a
:10660c00028240004220a80085824c004200a90072
:10661c004220ae004200a8000482d300a7018000f3
:10662c000503780004027800a6018800004a78006f
:10663c00a701880034a020009e004200610ab80027
:10664c00848fd2008582d2000402780004f0a1006d
:10665c0003c0250033b79a000600200046b79a0005
:10666c00970180003eb49200ceb492000801d00095
:10667c008401d000030241004220a80085824c0016
:10668c004200a9004220ae004200a8000482d300c0
:10669c000503780096018800040278001442780003
:1066ac00970188000440e800610ab800848fd2008a
:1066bc008582d2000402780004f0a10006c02500f7
:1066cc0056b79a000700200067b79a005eb4920094
:1066dc00eeb492008800d0000401d0000282400089
:1066ec004220a80085824c004200a9004220ae0046
:1066fc004200a8000482d300a701800005037800a3
:10670c0004027800a6018800004a7800a7018800de
:10671c0044a020009e004200610ab800848fd20081
:10672c008582d2000402780004f0a10003c0250089
:10673c0073b79a000600200006bf9a0097018000ec
:10674c007eb492008ebc92000801d0008401d0006f
:10675c00030241004220a80085824c004200a9009f
:10676c004220ae004200a8000482d300050378004a
:10677c009601880004027800144278009701880082
:10678c000440e800610ab800848fd2008582d200f0
:10679c000402780004f0a10006c0250016bf9a0080
:1067ac000700200027bf9a001ebc9200aebc9200ce
:1067bc008800d0000401d000028240004220a800d2
:1067cc0085824c004200a9004220ae004200a80085
:1067dc000482d300a701800005037800040278002e
:1067ec00a6018800004a7800a701880054a0200068
:1067fc009e004200610ab800848fd2008582d200cc
:10680c000402780004f0a10003c0250033bf9a00f5
:10681c000600200046bf9a00970180003ebc920003
:10682c00cebc92000801d0008401d00003024100cc
:10683c004220a80085824c004200a9004220ae00f4
:10684c004200a8000482d30005037800960188005a
:10685c000402780014427800970188000440e80094
:10686c00610ab800848fd2008582d20004027800bd
:10687c0004f0a10006c0250056bf9a0007002000b6
:10688c0067bf9a005ebc9200eebc92008800d000fc
:10689c000401d000028240004220a80085824c00f6
:1068ac004200a9004220ae004200a8000482d3009e
:1068bc00a70180000503780004027800a601880077
:1068cc00004a7800a701880064a020009e004200c6
:1068dc00610ab800848fd2008582d200040278004d
:1068ec0004f0a10003c0250073bf9a00060020002d
:1068fc0006079b00970180007ebc92008e049300db
:10690c000801d0008401d000030241004220a800fd
:10691c0085824c004200a9004220ae004200a80033
:10692c000482d300050378009601880004027800e5
:10693c0014427800970188000440e800610ab8000e
:10694c00848fd2008582d2000402780004f0a1006a
:10695c0006c0250016079b000700200027079b0098
:10696c001e049300ae0493008800d0000401d000f4
:10697c00028240004220a80085824c004200a900ff
:10698c004220ae004200a8000482d300a701800080
:10699c000503780004027800a6018800004a7800fc
:1069ac00a701880074a020009e004200610ab80074
:1069bc00848fd2008582d2000402780004f0a100fa
:1069cc0003c0250033079b000600200046079b00f0
:1069dc00970180003e049300ce0493000801d00080
:1069ec008401d000030241004220a80085824c00a3
:1069fc004200a9004220ae004200a8000482d3004d
:106a0c00050378009601880004027800144278008f
:106a1c00970188000440e800610ab800848fd20016
:106a2c008582d2000402780004f0a10006c0250083
:106a3c0056079b000700200067079b005e0493002d
:106a4c00ee0493008800d0000401d00002824000c4
:106a5c004220a80085824c004200a9004220ae00d2
:106a6c004200a8000482d300a7018000050378002f
:106a7c0004027800a6018800004a7800a70188006b
:106a8c0004aa20009e004200610ab800848fd20044
:106a9c008582d2000402780004f0a10003c0250016
:106aac0073079b0006002000060f9b0097018000d7
:106abc007e0493008e0c93000801d0008401d0005a
:106acc00030241004220a80085824c004200a9002c
:106adc004220ae004200a8000482d30005037800d7
:106aec00960188000402780014427800970188000f
:106afc000440e800610ab800848fd2008582d2007d
:106b0c000402780004f0a10006c02500160f9b00bb
:106b1c0007002000270f9b001e0c9300ae0c930067
:106b2c008800d0000401d000028240004220a8005e
:106b3c0085824c004200a9004220ae004200a80011
:106b4c000482d300a70180000503780004027800ba
:106b5c00a6018800004a7800a701880014aa20002a
:106b6c009e004200610ab800848fd2008582d20058
:106b7c000402780004f0a10003c02500330f9b0031
:106b8c0006002000460f9b00970180003e0c9300ee
:106b9c00ce0c93000801d0008401d0000302410008
:106bac004220a80085824c004200a9004220ae0081
:106bbc004200a8000482d3000503780096018800e7
:106bcc000402780014427800970188000440e80021
:106bdc00610ab800848fd2008582d200040278004a
:106bec0004f0a10006c02500560f9b0007002000f2
:106bfc00670f9b005e0c9300ee0c93008800d00096
:106c0c000401d000028240004220a80085824c0082
:106c1c004200a9004220ae004200a8000482d3002a
:106c2c00a70180000503780004027800a601880003
:106c3c00004a7800a701880024aa20009e00420088
:106c4c00610ab800848fd2008582d20004027800d9
:106c5c0004f0a10003c02500730f9b000600200068
:106c6c0006179b00970180007e0c93008e149300f6
:106c7c000801d0008401d000030241004220a8008a
:106c8c0085824c004200a9004220ae004200a800c0
:106c9c000482d30005037800960188000402780072
:106cac0014427800970188000440e800610ab8009b
:106cbc00848fd2008582d2000402780004f0a100f7
:106ccc0006c0250016179b000700200027179b0005
:106cdc001e149300ae1493008800d0000401d00061
:106cec00028240004220a80085824c004200a9008c
:106cfc004220ae004200a8000482d300a70180000d
:106d0c000503780004027800a6018800004a780088
:106d1c00a701880034aa20009e004200610ab80036
:106d2c00848fd2008582d2000402780004f0a10086
:106d3c0003c0250033179b000600200046179b005c
:106d4c00970180003e149300ce1493000801d000ec
:106d5c008401d000030241004220a80085824c002f
:106d6c004200a9004220ae004200a8000482d300d9
:106d7c00050378009601880004027800144278001c
:106d8c00970188000440e800610ab800848fd200a3
:106d9c008582d2000402780004f0a10006c0250010
:106dac0056179b000700200067179b005e1493008a
:106dbc00ee1493008800d0000401d0000282400041
:106dcc004220a80085824c004200a9004220ae005f
:106ddc004200a8000482d300a701800005037800bc
:106dec0004027800a6018800004a7800a7018800f8
:106dfc0044aa20009e004200610ab800848fd20091
:106e0c008582d2000402780004f0a10003c02500a2
:106e1c0073179b0006002000061f9b009701800043
:106e2c007e1493008e1c93000801d0008401d000c6
:106e3c00030241004220a80085824c004200a900b8
:106e4c004220ae004200a8000482d3000503780063
:106e5c00960188000402780014427800970188009b
:106e6c000440e800610ab800848fd2008582d20009
:106e7c000402780004f0a10006c02500161f9b0038
:106e8c0007002000271f9b001e1c9300ae1c9300c4
:106e9c008800d0000401d000028240004220a800eb
:106eac0085824c004200a9004220ae004200a8009e
:106ebc000482d300a7018000050378000402780047
:106ecc00a6018800004a7800a701880054aa200077
:106edc009e004200610ab800848fd2008582d200e5
:106eec000402780004f0a10003c02500331f9b00ae
:106efc0006002000461f9b00970180003e1c93005b
:106f0c00ce1c93000801d0008401d0000302410084
:106f1c004220a80085824c004200a9004220ae000d
:106f2c004200a8000482d300050378009601880073
:106f3c000402780014427800970188000440e800ad
:106f4c00610ab800848fd2008582d20004027800d6
:106f5c0004f0a10006c02500561f9b00070020006e
:106f6c00671f9b005e1c9300ee1c93008800d000f2
:106f7c000401d000028240004220a80085824c000f
:106f8c004200a9004220ae004200a8000482d300b7
:106f9c00a70180000503780004027800a601880090
:106fac00004a7800a701880064aa20009e004200d5
:106fbc00610ab800848fd2008582d2000402780066
:106fcc0004f0a10003c02500731f9b0006002000e5
:106fdc0006279b00970180007e1c93008e24930053
:106fec000801d0008401d000030241004220a80017
:106ffc0085824c004200a9004220ae004200a8004d
:10700c000482d300050378009601880004027800fe
:10701c0014427800970188000440e800610ab80027
:10702c00848fd2008582d2000402780004f0a10083
:10703c0006c0250016279b000700200027279b0071
:10704c001e249300ae2493008800d0000401d000cd
:10705c00028240004220a80085824c004200a90018
:10706c004220ae004200a8000482d300a701800099
:10707c000503780004027800a6018800004a780015
:10708c00a701880074aa20009e004200610ab80083
:10709c00848fd2008582d2000402780004f0a10013
:1070ac0003c0250033279b000600200046279b00c9
:1070bc00970180003e249300ce2493000801d00059
:1070cc008401d000030241004220a80085824c00bc
:1070dc004200a9004220ae004200a8000482d30066
:1070ec0005037800960188000402780014427800a9
:1070fc00970188000440e800610ab800848fd20030
:10710c008582d2000402780004f0a10006c025009c
:10711c0056279b000700200067279b005e249300e6
:10712c00ee2493008800d0000401d00002824000bd
:10713c004220a80085824c004200a9004220ae00eb
:10714c004200a8000482d300a70180000503780048
:10715c0004027800a6018800004a7800a701880084
:10716c0004b420009e004200610ab800848fd20053
:10717c008582d2000402780004f0a10003c025002f
:10718c0073279b0006002000062f9b0097018000b0
:10719c007e2493008e2c93000801d0008401d00033
:1071ac00030241004220a80085824c004200a90045
:1071bc004220ae004200a8000482d30005037800f0
:1071cc009601880004027800144278009701880028
:1071dc000440e800610ab800848fd2008582d20096
:1071ec000402780004f0a10006c02500162f9b00b5
:1071fc0007002000272f9b001e2c9300ae2c930021
:10720c008800d0000401d000028240004220a80077
:10721c0085824c004200a9004220ae004200a8002a
:10722c000482d300a70180000503780004027800d3
:10723c00a6018800004a7800a701880014b4200039
:10724c009e004200610ab800848fd2008582d20071
:10725c000402780004f0a10003c02500332f9b002a
:10726c0006002000462f9b00970180003e2c9300c7
:10727c00ce2c93000801d0008401d0000302410001
:10728c004220a80085824c004200a9004220ae009a
:10729c004200a8000482d300050378009601880000
:1072ac000402780014427800970188000440e8003a
:1072bc00610ab800848fd2008582d2000402780063
:1072cc0004f0a10006c02500562f9b0007002000eb
:1072dc00672f9b005e2c9300ee2c93008800d0004f
:1072ec000401d000028240004220a80085824c009c
:1072fc004200a9004220ae004200a8000482d30044
:10730c00a70180000503780004027800a60188001c
:10731c00004a7800a701880024b420009e00420097
:10732c00610ab800848fd2008582d20004027800f2
:10733c0004f0a10003c02500732f9b000600200061
:10734c0006379b00970180007e2c93008e349300af
:10735c000801d0008401d000030241004220a800a3
:10736c0085824c004200a9004220ae004200a800d9
:10737c000482d3000503780096018800040278008b
:10738c0014427800970188000440e800610ab800b4
:10739c00848fd2008582d2000402780004f0a10010
:1073ac0006c0250016379b000700200027379b00de
:1073bc001e349300ae3493008800d0000401d0003a
:1073cc00028240004220a80085824c004200a900a5
:1073dc004220ae004200a8000482d300a701800026
:1073ec000503780004027800a6018800004a7800a2
:1073fc00a701880034b420009e004200610ab80046
:10740c00848fd2008582d2000402780004f0a1009f
:10741c0003c0250033379b000600200046379b0035
:10742c00970180003e349300ce3493000801d000c5
:10743c008401d000030241004220a80085824c0048
:10744c004200a9004220ae004200a8000482d300f2
:10745c000503780096018800040278001442780035
:10746c00970188000440e800610ab800848fd200bc
:10747c008582d2000402780004f0a10006c0250029
:10748c0056379b000700200067379b005e34930043
:10749c00ee3493008800d0000401d000028240003a
:1074ac004220a80085824c004200a9004220ae0078
:1074bc004200a8000482d300a701800005037800d5
:1074cc0004027800a6018800004a7800a701880011
:1074dc0044b420009e004200610ab800848fd200a0
:1074ec008582d2000402780004f0a10003c02500bc
:1074fc0073379b0006002000063f9b00970180001d
:10750c007e3493008e3c93000801d0008401d0009f
:10751c00030241004220a80085824c004200a900d1
:10752c004220ae004200a8000482d300050378007c
:10753c0096018800040278001442780097018800b4
:10754c000440e800610ab800848fd2008582d20022
:10755c000402780004f0a10006c02500163f9b0031
:10756c0007002000273f9b001e3c9300ae3c93007d
:10757c008800d0000401d000028240004220a80004
:10758c0085824c004200a9004220ae004200a800b7
:10759c000482d300a7018000050378000402780060
:1075ac00a6018800004a7800a701880054b4200086
:1075bc009e004200610ab800848fd2008582d200fe
:1075cc000402780004f0a10003c02500333f9b00a7
:1075dc0006002000463f9b00970180003e3c930034
:1075ec00ce3c93000801d0008401d000030241007e
:1075fc004220a80085824c004200a9004220ae0027
:10760c004200a8000482d30005037800960188008c
:10761c000402780014427800970188000440e800c6
:10762c00610ab800848fd2008582d20004027800ef
:10763c0004f0a10006c02500563f9b000700200067
:10764c00673f9b005e3c9300ee3c93008800d000ab
:10765c000401d000028240004220a80085824c0028
:10766c004200a9004220ae004200a8000482d300d0
:10767c00a70180000503780004027800a6018800a9
:10768c00004a7800a701880064b420009e004200e4
:10769c00610ab800848fd2008582d200040278007f
:1076ac0004f0a10003c02500733f9b0006002000de
:1076bc0006879b00970180007e3c93008e8493008c
:1076cc000801d0008401d000030241004220a80030
:1076dc0085824c004200a9004220ae004200a80066
:1076ec000482d30005037800960188000402780018
:1076fc0014427800970188000440e800610ab80041
:10770c00848fd2008582d2000402780004f0a1009c
:10771c0006c0250016879b000700200027879b00ca
:10772c001e849300ae8493008800d0000401d00026
:10773c00028240004220a80085824c004200a90031
:10774c004220ae004200a8000482d300a7018000b2
:10775c000503780004027800a6018800004a78002e
:10776c00a701880074b420009e004200610ab80092
:10777c00848fd2008582d2000402780004f0a1002c
:10778c0003c0250033879b000600200046879b0022
:10779c00970180003e849300ce8493000801d000b2
:1077ac008401d000030241004220a80085824c00d5
:1077bc004200a9004220ae004200a8000482d3007f
:1077cc0005037800960188000402780014427800c2
:1077dc00970188000440e800610ab800848fd20049
:1077ec008582d2000402780004f0a10006c02500b6
:1077fc0056879b000700200067879b005e849300e0
:10780c00ee8493008800d0000401d0000282400076
:10781c004220a80085824c004200a9004220ae0004
:10782c004200a8000482d300a70180000503780061
:10783c0004027800a6018800004a7800a70188009d
:10784c0004be20009e004200610ab800848fd20062
:10785c008582d2000402780004f0a10003c0250048
:10786c0073879b0006002000068f9b009701800009
:10787c007e8493008e8c93000801d0008401d0008c
:10788c00030241004220a80085824c004200a9005e
:10789c004220ae004200a8000482d3000503780009
:1078ac009601880004027800144278009701880041
:1078bc000440e800610ab800848fd2008582d200af
:1078cc000402780004f0a10006c02500168f9b006e
:1078dc0007002000278f9b001e8c9300ae8c93001a
:1078ec008800d0000401d000028240004220a80091
:1078fc0085824c004200a9004220ae004200a80044
:10790c000482d300a70180000503780004027800ec
:10791c00a6018800004a7800a701880014be200048
:10792c009e004200610ab800848fd2008582d2008a
:10793c000402780004f0a10003c02500338f9b00e3
:10794c0006002000468f9b00970180003e8c930020
:10795c00ce8c93000801d0008401d00003024100ba
:10796c004220a80085824c004200a9004220ae00b3
:10797c004200a8000482d300050378009601880019
:10798c000402780014427800970188000440e80053
:10799c00610ab800848fd2008582d200040278007c
:1079ac0004f0a10006c02500568f9b0007002000a4
:1079bc00678f9b005e8c9300ee8c93008800d00048
:1079cc000401d000028240004220a80085824c00b5
:1079dc004200a9004220ae004200a8000482d3005d
:1079ec00a70180000503780004027800a601880036
:1079fc00004a7800a701880024be20009e004200a7
:107a0c00610ab800848fd2008582d200040278000b
:107a1c0004f0a10003c02500738f9b00060020001a
:107a2c0006979b00970180007e8c93008e949300a8
:107a3c000801d0008401d000030241004220a800bc
:107a4c0085824c004200a9004220ae004200a800f2
:107a5c000482d300050378009601880004027800a4
:107a6c0014427800970188000440e800610ab800cd
:107a7c00848fd2008582d2000402780004f0a10029
:107a8c0006c0250016979b000700200027979b0037
:107a9c001e949300ae9493008800d0000401d00093
:107aac00028240004220a80085824c004200a900be
:107abc004220ae004200a8000482d300a70180003f
:107acc000503780004027800a6018800004a7800bb
:107adc00a701880034be20009e004200610ab80055
:107aec00848fd2008582d2000402780004f0a100b9
:107afc0003c0250033979b000600200046979b008f
:107b0c00970180003e949300ce9493000801d0001e
:107b1c008401d000030241004220a80085824c0061
:107b2c004200a9004220ae004200a8000482d3000b
:107b3c00050378009601880004027800144278004e
:107b4c00970188000440e800610ab800848fd200d5
:107b5c008582d2000402780004f0a10006c0250042
:107b6c0056979b000700200067979b005e9493003c
:107b7c00ee9493008800d0000401d00002824000f3
:107b8c004220a80085824c004200a9004220ae0091
:107b9c004200a8000482d300a701800005037800ee
:107bac0004027800a6018800004a7800a70188002a
:107bbc0044be20009e004200610ab800848fd200af
:107bcc008582d2000402780004f0a10003c02500d5
:107bdc0073979b0006002000069f9b009701800076
:107bec007e9493008e9c93000801d0008401d000f9
:107bfc00030241004220a80085824c004200a900eb
:107c0c004220ae004200a8000482d3000503780095
:107c1c0096018800040278001442780097018800cd
:107c2c000440e800610ab800848fd2008582d2003b
:107c3c000402780004f0a10006c02500169f9b00ea
:107c4c0007002000279f9b001e9c9300ae9c930076
:107c5c008800d0000401d000028240004220a8001d
:107c6c0085824c004200a9004220ae004200a800d0
:107c7c000482d300a7018000050378000402780079
:107c8c00a6018800004a7800a701880054be200095
:107c9c009e004200610ab800848fd2008582d20017
:107cac000402780004f0a10003c02500339f9b0060
:107cbc0006002000469f9b00970180003e9c93008d
:107ccc00ce9c93000801d0008401d0000302410037
:107cdc004220a80085824c004200a9004220ae0040
:107cec004200a8000482d3000503780096018800a6
:107cfc000402780014427800970188000440e800e0
:107d0c00610ab800848fd2008582d2000402780008
:107d1c0004f0a10006c02500569f9b000700200020
:107d2c00679f9b005e9c9300ee9c93008800d000a4
:107d3c000401d000028240004220a80085824c0041
:107d4c004200a9004220ae004200a8000482d300e9
:107d5c00a70180000503780004027800a6018800c2
:107d6c00004a7800a701880064be20009e004200f3
:107d7c00610ab800848fd2008582d2000402780098
:107d8c0004f0a10003c02500739f9b000600200097
:107d9c0006a79b00970180007e9c93008ea4930005
:107dac000801d0008401d000030241004220a80049
:107dbc0085824c004200a9004220ae004200a8007f
:107dcc000482d30005037800960188000402780031
:107ddc0014427800970188000440e800610ab8005a
:107dec00848fd2008582d2000402780004f0a100b6
:107dfc0006c0250016a79b000700200027a79b00a4
:107e0c001ea49300aea493008800d0000401d000ff
:107e1c00028240004220a80085824c004200a9004a
:107e2c004220ae004200a8000482d300a7018000cb
:107e3c000503780004027800a6018800004a780047
:107e4c00a701880074be20009e004200610ab800a1
:107e5c00848fd2008582d2000402780004f0a10045
:107e6c0003c0250033a79b000600200046a79b00fb
:107e7c00970180003ea49300cea493000801d0008b
:107e8c008401d000030241004220a80085824c00ee
:107e9c004200a9004220ae004200a8000482d30098
:107eac0005037800960188000402780014427800db
:107ebc00970188000440e800610ab800848fd20062
:107ecc008582d2000402780004f0a10006c02500cf
:107edc0056a79b000700200067a79b005ea4930099
:107eec00eea493008800d0000401d0000282400070
:107efc004220a80085824c004200a9004220ae001e
:107f0c004200a8000482d300a7018000050378007a
:107f1c0004027800a6018800004a7800a7018800b6
:107f2c0004c820009e004200610ab800848fd20071
:107f3c008582d2000402780004f0a10003c0250061
:107f4c0073a79b000600200006af9b0097018000e2
:107f5c007ea493008eac93000801d0008401d00065
:107f6c00030241004220a80085824c004200a90077
:107f7c004220ae004200a8000482d3000503780022
:107f8c00960188000402780014427800970188005a
:107f9c000440e800610ab800848fd2008582d200c8
:107fac000402780004f0a10006c0250016af9b0067
:107fbc000700200027af9b001eac9300aeac9300d3
:107fcc008800d0000401d000028240004220a800aa
:107fdc0085824c004200a9004220ae004200a8005d
:107fec000482d300a7018000050378000402780006
:107ffc00a6018800004a7800a701880014c8200058
:10800c009e004200610ab800848fd2008582d200a3
:10801c000402780004f0a10003c0250033af9b00dc
:10802c000600200046af9b00970180003eac9300f9
:10803c00ceac93000801d0008401d00003024100b3
:10804c004220a80085824c004200a9004220ae00cc
:10805c004200a8000482d300050378009601880032
:10806c000402780014427800970188000440e8006c
:10807c00610ab800848fd2008582d2000402780095
:10808c0004f0a10006c0250056af9b00070020009d
:10809c0067af9b005eac9300eeac93008800d00001
:1080ac000401d000028240004220a80085824c00ce
:1080bc004200a9004220ae004200a8000482d30076
:1080cc00a70180000503780004027800a60188004f
:1080dc00004a7800a701880024c820009e004200b6
:1080ec00610ab800848fd2008582d2000402780025
:1080fc0004f0a10003c0250073af9b000600200014
:10810c0006b79b00970180007eac93008eb4930061
:10811c000801d0008401d000030241004220a800d5
:10812c0085824c004200a9004220ae004200a8000b
:10813c000482d300050378009601880004027800bd
:10814c0014427800970188000440e800610ab800e6
:10815c00848fd2008582d2000402780004f0a10042
:10816c0006c0250016b79b000700200027b79b0010
:10817c001eb49300aeb493008800d0000401d0006c
:10818c00028240004220a80085824c004200a900d7
:10819c004220ae004200a8000482d300a701800058
:1081ac000503780004027800a6018800004a7800d4
:1081bc00a701880034c820009e004200610ab80064
:1081cc00848fd2008582d2000402780004f0a100d2
:1081dc0003c0250033b79b000600200046b79b0068
:1081ec00970180003eb49300ceb493000801d000f8
:1081fc008401d000030241004220a80085824c007b
:10820c004200a9004220ae004200a8000482d30024
:10821c000503780096018800040278001442780067
:10822c00970188000440e800610ab800848fd200ee
:10823c008582d2000402780004f0a10006c025005b
:10824c0056b79b000700200067b79b005eb49300f5
:10825c00eeb493008800d0000401d00002824000ec
:10826c004220a80085824c004200a9004220ae00aa
:10827c004200a8000482d300a70180000503780007
:10828c0004027800a6018800004a7800a701880043
:10829c0044c820009e004200610ab800848fd200be
:1082ac008582d2000402780004f0a10003c02500ee
:1082bc0073b79b000600200006bf9b00970180004f
:1082cc007eb493008ebc93000801d0008401d000d2
:1082dc00030241004220a80085824c004200a90004
:1082ec004220ae004200a8000482d30005037800af
:1082fc0096018800040278001442780097018800e7
:10830c000440e800610ab800848fd2008582d20054
:10831c000402780004f0a10006c0250016bf9b00e3
:10832c000700200027bf9b001ebc9300aebc93002f
:10833c008800d0000401d000028240004220a80036
:10834c0085824c004200a9004220ae004200a800e9
:10835c000482d300a7018000050378000402780092
:10836c00a6018800004a7800a701880054c82000a4
:10837c009e004200610ab800848fd2008582d20030
:10838c000402780004f0a10003c0250033bf9b0059
:10839c000600200046bf9b00970180003ebc930066
:1083ac00cebc93000801d0008401d0000302410030
:1083bc004220a80085824c004200a9004220ae0059
:1083cc004200a8000482d3000503780096018800bf
:1083dc000402780014427800970188000440e800f9
:1083ec00610ab800848fd2008582d2000402780022
:1083fc0004f0a10006c0250056bf9b00070020001a
:10840c0067bf9b005ebc9300eebc93008800d0005d
:10841c000401d000028240004220a80085824c005a
:10842c004200a9004220ae004200a8000482d30002
:10843c00a70180000503780004027800a6018800db
:10844c00004a7800a701880064c820009e00420002
:10845c00610ab800848fd2008582d20004027800b1
:10846c0004f0a10003c0250073bf9b00080020008e
:10847c00064020000e03430086037800880b78002a
:10848c0097018000e33f20008e8141001301be0064
:10849c000203d0000404d000080243004220a800cc
:1084ac00858249004200a9004220ae004200a8008b
:1084bc000482d3000503780096018800040278003a
:1084cc0014427800970188000440e800610ab80063
:1084dc00848fd2008582d2000402780004f0a100bf
:1084ec0002c02500294020008e84440089007800b9
:1084fc008208780007002000434020008e81410054
:10850c0003037800070b7800294020008e84440078
:10851c001904be008800d0000401d0000282400083
:10852c004220a80085824c004200a9004220ae00e7
:10853c004200a8000482d300a70180000503780044
:10854c0004027800a6018800004a7800a701880080
:10855c0074c820009e004200610ab800848fd200cb
:10856c008582d2000402780004f0a10007c0250027
:10857c00634020008e81410003037800070b7800d4
:10858c0002002000884020000e044400880478007b
:10859c00820c780097018000694020008e84440092
:1085ac001904be000801d0008401d0000302410070
:1085bc004220a80085824c004200a9004220ae0057
:1085cc004200a8000482d3000503780096018800bd
:1085dc000402780014427800970188000440e800f7
:1085ec00610ab800848fd2008582d2000402780020
:1085fc0004f0a10008c02500a64020000e03430093
:10860c0086037800880b780002002000c940200007
:10861c008e8444008900780082087800a7402000ee
:10862c008e8343001703be000604d0008404d000e0
:10863c00090244004220a80085824b004200a90098
:10864c004220ae004200a8000482d300a7018000a3
:10865c000503780004027800a6018800004a78001f
:10866c00a701880004d220009e004200610ab800d5
:10867c00848fd2008582d2000402780004f0a1001d
:10868c0006c02500e24020000e0141008201780066
:10869c008609780009002000074120008e834300e2
:1086ac0007047800090c780097018000e340200053
:1086bc008e8141001301be000203d0000404d000df
:1086cc00080243004220a800858249004200a9000c
:1086dc004220ae004200a8000482d30005037800bb
:1086ec0096018800040278001442780097018800f3
:1086fc000440e800610ab800848fd2008582d20061
:10870c000402780004f0a10002c0250029412000d9
:10871c008e844400890078008208780007002000cd
:10872c00434120008e81410003037800070b780041
:10873c00294120008e8444001904be008800d0001a
:10874c000401d000028240004220a80085824c0027
:10875c004200a9004220ae004200a8000482d300cf
:10876c00a70180000503780004027800a6018800a8
:10877c00004a7800a701880014d220009e00420015
:10878c00610ab800848fd2008582d200040278007e
:10879c0004f0a10007c02500634120008e81410038
:1087ac0003037800070b78000200200088412000aa
:1087bc000e04440088047800820c78009701800035
:1087cc00694120008e8444001904be000801d000c9
:1087dc008401d000030241004220a80085824c0095
:1087ec004200a9004220ae004200a8000482d3003f
:1087fc000503780096018800040278001442780082
:10880c00970188000440e800610ab800848fd20008
:10881c008582d2000402780004f0a10008c0250073
:10882c00a64120000e03430086037800880b7800d5
:10883c0002002000c94120008e8444008900780089
:10884c0082087800a74120008e8343001703be00e6
:10885c000604d0008404d000090244004220a80081
:10886c0085824b004200a9004220ae004200a800c5
:10887c000482d300a701800005037800040278006d
:10888c00a6018800004a7800a701880024d22000a5
:10889c009e004200610ab800848fd2008582d2000b
:1088ac000402780004f0a10006c02500e24120007b
:1088bc000e01410082017800860978000900200031
:1088cc00074220008e83430007047800090c7800cf
:1088dc0097018000e34120008e8141001301be000e
:1088ec000203d0000404d000080243004220a80078
:1088fc00858249004200a9004220ae004200a80037
:10890c000482d300050378009601880004027800e5
:10891c0014427800970188000440e800610ab8000e
:10892c00848fd2008582d2000402780004f0a1006a
:10893c0002c02500294220008e8444008900780062
:10894c008208780007002000434220008e814100fd
:10895c0003037800070b7800294220008e84440022
:10896c001904be008800d0000401d000028240002f
:10897c004220a80085824c004200a9004220ae0093
:10898c004200a8000482d300a701800005037800f0
:10899c0004027800a6018800004a7800a70188002c
:1089ac0034d220009e004200610ab800848fd200ad
:1089bc008582d2000402780004f0a10007c02500d3
:1089cc00634220008e81410003037800070b78007e
:1089dc0002002000884220000e0444008804780025
:1089ec00820c780097018000694220008e8444003c
:1089fc001904be000801d0008401d000030241001c
:108a0c004220a80085824c004200a9004220ae0002
:108a1c004200a8000482d300050378009601880068
:108a2c000402780014427800970188000440e800a2
:108a3c00610ab800848fd2008582d20004027800cb
:108a4c0004f0a10008c02500a64220000e0343003c
:108a5c0086037800880b780002002000c9422000b1
:108a6c008e8444008900780082087800a742200098
:108a7c008e8343001703be000604d0008404d0008c
:108a8c00090244004220a80085824b004200a90044
:108a9c004220ae004200a8000482d300a70180004f
:108aac000503780004027800a6018800004a7800cb
:108abc00a701880044d220009e004200610ab80041
:108acc00848fd2008582d2000402780004f0a100c9
:108adc0006c02500e24220000e0141008201780010
:108aec008609780009002000074320008e8343008c
:108afc0007047800090c780097018000e3422000fd
:108b0c008e8141001301be000203d0000404d0008a
:108b1c00080243004220a800858249004200a900b7
:108b2c004220ae004200a8000482d3000503780066
:108b3c00960188000402780014427800970188009e
:108b4c000440e800610ab800848fd2008582d2000c
:108b5c000402780004f0a10002c025002943200083
:108b6c008e84440089007800820878000700200079
:108b7c00434320008e81410003037800070b7800eb
:108b8c00294320008e8444001904be008800d000c4
:108b9c000401d000028240004220a80085824c00d3
:108bac004200a9004220ae004200a8000482d3007b
:108bbc00a70180000503780004027800a601880054
:108bcc00004a7800a701880054d220009e00420081
:108bdc00610ab800848fd2008582d200040278002a
:108bec0004f0a10007c02500634320008e814100e2
:108bfc0003037800070b7800020020008843200054
:108c0c000e04440088047800820c780097018000e0
:108c1c00694320008e8444001904be000801d00072
:108c2c008401d000030241004220a80085824c0040
:108c3c004200a9004220ae004200a8000482d300ea
:108c4c00050378009601880004027800144278002d
:108c5c00970188000440e800610ab800848fd200b4
:108c6c008582d2000402780004f0a10008c025001f
:108c7c00a64320000e03430086037800880b78007f
:108c8c0002002000c94320008e8444008900780033
:108c9c0082087800a74320008e8343001703be0090
:108cac000604d0008404d000090244004220a8002d
:108cbc0085824b004200a9004220ae004200a80071
:108ccc000482d300a7018000050378000402780019
:108cdc00a6018800004a7800a701880064d2200011
:108cec009e004200610ab800848fd2008582d200b7
:108cfc000402780004f0a10006c02500e243200025
:108d0c000e014100820178008609780009002000dc
:108d1c00074420008e83430007047800090c780078
:108d2c0097018000e34320008e8141001301be00b7
:108d3c000203d0000404d000080243004220a80023
:108d4c00858249004200a9004220ae004200a800e2
:108d5c000482d30005037800960188000402780091
:108d6c0014427800970188000440e800610ab800ba
:108d7c00848fd2008582d2000402780004f0a10016
:108d8c0002c02500294420008e844400890078000c
:108d9c008208780007002000434420008e814100a7
:108dac0003037800070b7800294420008e844400cc
:108dbc001904be008800d0000401d00002824000db
:108dcc004220a80085824c004200a9004220ae003f
:108ddc004200a8000482d300a7018000050378009c
:108dec0004027800a6018800004a7800a7018800d8
:108dfc0074d220009e004200610ab800848fd20019
:108e0c008582d2000402780004f0a10007c025007e
:108e1c00634420008e81410003037800070b780027
:108e2c0002002000884420000e04440088047800ce
:108e3c00820c780097018000694420008e844400e5
:108e4c001904be000801d0008401d00003024100c7
:108e5c004220a80085824c004200a9004220ae00ae
:108e6c004200a8000482d300050378009601880014
:108e7c000402780014427800970188000440e8004e
:108e8c00610ab800848fd2008582d2000402780077
:108e9c0004f0a10008c02500a64420000e034300e6
:108eac0086037800880b780002002000c94420005b
:108ebc008e8444008900780082087800a744200042
:108ecc008e8343001703be000604d0008404d00038
:108edc00090244004220a80085824b004200a900f0
:108eec004220ae004200a8000482d300a7018000fb
:108efc000503780004027800a6018800004a780077
:108f0c00a701880004dc20009e004200610ab80022
:108f1c00848fd2008582d2000402780004f0a10074
:108f2c0006c02500e24420000e01410082017800b9
:108f3c008609780009002000074520008e83430035
:108f4c0007047800090c780097018000e3442000a6
:108f5c008e8141001301be000203d0000404d00036
:108f6c00080243004220a800858249004200a90063
:108f7c004220ae004200a8000482d3000503780012
:108f8c00960188000402780014427800970188004a
:108f9c000440e800610ab800848fd2008582d200b8
:108fac000402780004f0a10002c02500294520002d
:108fbc008e84440089007800820878000700200025
:108fcc00434520008e81410003037800070b780095
:108fdc00294520008e8444001904be008800d0006e
:108fec000401d000028240004220a80085824c007f
:108ffc004200a9004220ae004200a8000482d30027
:10900c00a70180000503780004027800a6018800ff
:10901c00004a7800a701880014dc20009e00420062
:10902c00610ab800848fd2008582d20004027800d5
:10903c0004f0a10007c02500634520008e8141008b
:10904c0003037800070b78000200200088452000fd
:10905c000e04440088047800820c7800970180008c
:10906c00694520008e8444001904be000801d0001c
:10907c008401d000030241004220a80085824c00ec
:10908c004200a9004220ae004200a8000482d30096
:10909c0005037800960188000402780014427800d9
:1090ac00970188000440e800610ab800848fd20060
:1090bc008582d2000402780004f0a10008c02500cb
:1090cc00a64520000e03430086037800880b780029
:1090dc0002002000c94520008e84440089007800dd
:1090ec0082087800a74520008e8343001703be003a
:1090fc000604d0008404d000090244004220a800d9
:10910c0085824b004200a9004220ae004200a8001c
:10911c000482d300a70180000503780004027800c4
:10912c00a6018800004a7800a701880024dc2000f2
:10913c009e004200610ab800848fd2008582d20062
:10914c000402780004f0a10006c02500e2452000ce
:10915c000e01410082017800860978000900200088
:10916c00074620008e83430007047800090c780022
:10917c0097018000e34520008e8141001301be0061
:10918c000203d0000404d000080243004220a800cf
:10919c00858249004200a9004220ae004200a8008e
:1091ac000482d3000503780096018800040278003d
:1091bc0014427800970188000440e800610ab80066
:1091cc00848fd2008582d2000402780004f0a100c2
:1091dc0002c02500294620008e84440089007800b6
:1091ec008208780007002000434620008e81410051
:1091fc0003037800070b7800294620008e84440076
:10920c001904be008800d0000401d0000282400086
:10921c004220a80085824c004200a9004220ae00ea
:10922c004200a8000482d300a70180000503780047
:10923c0004027800a6018800004a7800a701880083
:10924c0034dc20009e004200610ab800848fd200fa
:10925c008582d2000402780004f0a10007c025002a
:10926c00634620008e81410003037800070b7800d1
:10927c0002002000884620000e0444008804780078
:10928c00820c780097018000694620008e8444008f
:10929c001904be000801d0008401d0000302410073
:1092ac004220a80085824c004200a9004220ae005a
:1092bc004200a8000482d3000503780096018800c0
:1092cc000402780014427800970188000440e800fa
:1092dc00610ab800848fd2008582d2000402780023
:1092ec0004f0a10008c02500a64620000e03430090
:1092fc0086037800880b780002002000c946200005
:10930c008e8444008900780082087800a7462000eb
:10931c008e8343001703be000604d0008404d000e3
:10932c00090244004220a80085824b004200a9009b
:10933c004220ae004200a8000482d300a7018000a6
:10934c000503780004027800a6018800004a780022
:10935c00a701880044dc20009e004200610ab8008e
:10936c00848fd2008582d2000402780004f0a10020
:10937c0006c02500e24620000e0141008201780063
:10938c008609780009002000074720008e834300df
:10939c0007047800090c780097018000e346200050
:1093ac008e8141001301be000203d0000404d000e2
:1093bc00080243004220a800858249004200a9000f
:1093cc004220ae004200a8000482d30005037800be
:1093dc0096018800040278001442780097018800f6
:1093ec000440e800610ab800848fd2008582d20064
:1093fc000402780004f0a10002c0250029472000d7
:10940c008e844400890078008208780007002000d0
:10941c00434720008e81410003037800070b78003e
:10942c00294720008e8444001904be008800d00017
:10943c000401d000028240004220a80085824c002a
:10944c004200a9004220ae004200a8000482d300d2
:10945c00a70180000503780004027800a6018800ab
:10946c00004a7800a701880054dc20009e004200ce
:10947c00610ab800848fd2008582d2000402780081
:10948c0004f0a10007c02500634720008e81410035
:10949c0003037800070b78000200200088472000a7
:1094ac000e04440088047800820c78009701800038
:1094bc00694720008e8444001904be000801d000c6
:1094cc008401d000030241004220a80085824c0098
:1094dc004200a9004220ae004200a8000482d30042
:1094ec000503780096018800040278001442780085
:1094fc00970188000440e800610ab800848fd2000c
:10950c008582d2000402780004f0a10008c0250076
:10951c00a64720000e03430086037800880b7800d2
:10952c0002002000c94720008e8444008900780086
:10953c0082087800a74720008e8343001703be00e3
:10954c000604d0008404d000090244004220a80084
:10955c0085824b004200a9004220ae004200a800c8
:10956c000482d300a7018000050378000402780070
:10957c00a6018800004a7800a701880064dc20005e
:10958c009e004200610ab800848fd2008582d2000e
:10959c000402780004f0a10006c02500e247200078
:1095ac000e01410082017800860978000900200034
:1095bc00074820008e83430007047800090c7800cc
:1095cc0097018000e34720008e8141001301be000b
:1095dc000203d0000404d000080243004220a8007b
:1095ec00858249004200a9004220ae004200a8003a
:1095fc000482d300050378009601880004027800e9
:10960c0014427800970188000440e800610ab80011
:10961c00848fd2008582d2000402780004f0a1006d
:10962c0002c02500294820008e844400890078005f
:10963c008208780007002000434820008e814100fa
:10964c0003037800070b7800294820008e8444001f
:10965c001904be008800d0000401d0000282400032
:10966c004220a80085824c004200a9004220ae0096
:10967c004200a8000482d300a701800005037800f3
:10968c0004027800a6018800004a7800a70188002f
:10969c0074dc20009e004200610ab800848fd20066
:1096ac008582d2000402780004f0a10007c02500d6
:1096bc00634820008e81410003037800070b78007b
:1096cc0002002000884820000e0444008804780022
:1096dc00820c780097018000694820008e84440039
:1096ec001904be000801d0008401d000030241001f
:1096fc004220a80085824c004200a9004220ae0006
:10970c004200a8000482d30005037800960188006b
:10971c000402780014427800970188000440e800a5
:10972c00610ab800848fd2008582d20004027800ce
:10973c0004f0a10008c02500a64820000e03430039
:10974c0086037800880b780002002000c9482000ae
:10975c008e8444008900780082087800a748200095
:10976c008e8343001703be000604d0008404d0008f
:10977c00090244004220a80085824b004200a90047
:10978c004220ae004200a8000482d300a701800052
:10979c000503780004027800a6018800004a7800ce
:1097ac00a701880014e620009e004200610ab80060
:1097bc00848fd2008582d2000402780004f0a100cc
:1097cc0006c02500e24820000e014100820178000d
:1097dc008609780009002000074920008e83430089
:1097ec0007047800090c780097018000e3482000fa
:1097fc008e8141001301be000203d0000404d0008e
:10980c00080243004220a800858249004200a900ba
:10981c004220ae004200a8000482d3000503780069
:10982c0096018800040278001442780097018800a1
:10983c000440e800610ab800848fd2008582d2000f
:10984c000402780004f0a10002c025002949200080
:10985c008e8444008900780082087800070020007c
:10986c00434920008e81410003037800070b7800e8
:10987c00294920008e8444001904be008800d000c1
:10988c000401d000028240004220a80085824c00d6
:10989c004200a9004220ae004200a8000482d3007e
:1098ac00a70180000503780004027800a601880057
:1098bc00004a7800a701880024e620009e004200a0
:1098cc00610ab800848fd2008582d200040278002d
:1098dc0004f0a10007c02500634920008e814100df
:1098ec0003037800070b7800020020008849200051
:1098fc000e04440088047800820c780097018000e4
:10990c00694920008e8444001904be000801d0006f
:10991c008401d000030241004220a80085824c0043
:10992c004200a9004220ae004200a8000482d300ed
:10993c000503780096018800040278001442780030
:10994c00970188000440e800610ab800848fd200b7
:10995c008582d2000402780004f0a10008c0250022
:10996c00a64920000e03430086037800880b78007c
:10997c0002002000c94920008e8444008900780030
:10998c0082087800a74920008e8343001703be008d
:10999c000604d0008404d000090244004220a80030
:1099ac0085824b004200a9004220ae004200a80074
:1099bc000482d300a701800005037800040278001c
:1099cc00a6018800004a7800a701880034e6200030
:1099dc009e004200610ab800848fd2008582d200ba
:1099ec000402780004f0a10006c02500e249200022
:1099fc000e014100820178008609780009002000e0
:109a0c00074a20008e83430007047800090c780075
:109a1c0097018000e34920008e8141001301be00b4
:109a2c000203d0000404d000080243004220a80026
:109a3c00858249004200a9004220ae004200a800e5
:109a4c000482d30005037800960188000402780094
:109a5c0014427800970188000440e800610ab800bd
:109a6c00848fd2008582d2000402780004f0a10019
:109a7c0002c02500294a20008e8444008900780009
:109a8c008208780007002000434a20008e814100a4
:109a9c0003037800070b7800294a20008e844400c9
:109aac001904be008800d0000401d00002824000de
:109abc004220a80085824c004200a9004220ae0042
:109acc004200a8000482d300a7018000050378009f
:109adc0004027800a6018800004a7800a7018800db
:109aec0044e620009e004200610ab800848fd20038
:109afc008582d2000402780004f0a10007c0250082
:109b0c00634a20008e81410003037800070b780024
:109b1c0002002000884a20000e04440088047800cb
:109b2c00820c780097018000694a20008e844400e2
:109b3c001904be000801d0008401d00003024100ca
:109b4c004220a80085824c004200a9004220ae00b1
:109b5c004200a8000482d300050378009601880017
:109b6c000402780014427800970188000440e80051
:109b7c00610ab800848fd2008582d200040278007a
:109b8c0004f0a10008c02500a64a20000e034300e3
:109b9c0086037800880b780002002000c94a200058
:109bac008e8444008900780082087800a74a20003f
:109bbc008e8343001703be000604d0008404d0003b
:109bcc00090244004220a80085824b004200a900f3
:109bdc004220ae004200a8000482d300a7018000fe
:109bec000503780004027800a6018800004a78007a
:109bfc00a701880054e620009e004200610ab800cc
:109c0c00848fd2008582d2000402780004f0a10077
:109c1c0006c02500e24a20000e01410082017800b6
:109c2c008609780009002000074b20008e83430032
:109c3c0007047800090c780097018000e34a2000a3
:109c4c008e8141001301be000203d0000404d00039
:109c5c00080243004220a800858249004200a90066
:109c6c004220ae004200a8000482d3000503780015
:109c7c00960188000402780014427800970188004d
:109c8c000440e800610ab800848fd2008582d200bb
:109c9c000402780004f0a10002c02500294b20002a
:109cac008e84440089007800820878000700200028
:109cbc00434b20008e81410003037800070b780092
:109ccc00294b20008e8444001904be008800d0006b
:109cdc000401d000028240004220a80085824c0082
:109cec004200a9004220ae004200a8000482d3002a
:109cfc00a70180000503780004027800a601880003
:109d0c00004a7800a701880064e620009e0042000b
:109d1c00610ab800848fd2008582d20004027800d8
:109d2c0004f0a10007c02500634b20008e81410088
:109d3c0003037800070b780002002000884b2000fa
:109d4c000e04440088047800820c7800970180008f
:109d5c00694b20008e8444001904be000801d00019
:109d6c008401d000030241004220a80085824c00ef
:109d7c004200a9004220ae004200a8000482d30099
:109d8c0005037800960188000402780014427800dc
:109d9c00970188000440e800610ab800848fd20063
:109dac008582d2000402780004f0a10008c02500ce
:109dbc00a64b20000e03430086037800880b780026
:109dcc0002002000c94b20008e84440089007800da
:109ddc0082087800a74b20008e8343001703be0037
:109dec000604d0008404d000090244004220a800dc
:109dfc0085824b004200a9004220ae004200a80020
:109e0c000482d300a70180000503780004027800c7
:109e1c00a6018800004a7800a701880014f02000f1
:109e2c009e004200610ab800848fd2008582d20065
:109e3c000402780004f0a10006c02500e24b2000cb
:109e4c000e0141008201780086097800090020008b
:109e5c00074c20008e83430007047800090c78001f
:109e6c0097018000e34b20008e8141001301be005e
:109e7c000203d0000404d000080243004220a800d2
:109e8c00858249004200a9004220ae004200a80091
:109e9c000482d30005037800960188000402780040
:109eac0014427800970188000440e800610ab80069
:109ebc00848fd2008582d2000402780004f0a100c5
:109ecc0002c02500294c20008e84440089007800b3
:109edc008208780007002000434c20008e8141004e
:109eec0003037800070b7800294c20008e84440073
:109efc001904be008800d0000401d000028240008a
:109f0c004220a80085824c004200a9004220ae00ed
:109f1c004200a8000482d300a7018000050378004a
:109f2c0004027800a6018800004a7800a701880086
:109f3c0024f020009e004200610ab800848fd200f9
:109f4c008582d2000402780004f0a10007c025002d
:109f5c00634c20008e81410003037800070b7800ce
:109f6c0002002000884c20000e0444008804780075
:109f7c00820c780097018000694c20008e8444008c
:109f8c001904be000801d0008401d0000302410076
:109f9c004220a80085824c004200a9004220ae005d
:109fac004200a8000482d3000503780096018800c3
:109fbc000402780014427800970188000440e800fd
:109fcc00610ab800848fd2008582d2000402780026
:109fdc0004f0a10008c02500a64c20000e0343008d
:109fec0086037800880b780002002000c94c200002
:109ffc008e8444008900780082087800a74c2000e9
:10a00c008e8343001703be000604d0008404d000e6
:10a01c00090244004220a80085824b004200a9009e
:10a02c004220ae004200a8000482d300a7018000a9
:10a03c000503780004027800a6018800004a780025
:10a04c00a701880034f020009e004200610ab8008d
:10a05c00848fd2008582d2000402780004f0a10023
:10a06c0006c02500e24c20000e0141008201780060
:10a07c008609780009002000074d20008e834300dc
:10a08c0007047800090c780097018000e34c20004d
:10a09c008e8141001301be000203d0000404d000e5
:10a0ac00080243004220a800858249004200a90012
:10a0bc004220ae004200a8000482d30005037800c1
:10a0cc0096018800040278001442780097018800f9
:10a0dc000440e800610ab800848fd2008582d20067
:10a0ec000402780004f0a10002c02500294d2000d4
:10a0fc008e844400890078008208780007002000d4
:10a10c00434d20008e81410003037800070b78003b
:10a11c00294d20008e8444001904be008800d00014
:10a12c000401d000028240004220a80085824c002d
:10a13c004200a9004220ae004200a8000482d300d5
:10a14c00a70180000503780004027800a6018800ae
:10a15c00004a7800a701880044f020009e004200cd
:10a16c00610ab800848fd2008582d2000402780084
:10a17c0004f0a10007c02500634d20008e81410032
:10a18c0003037800070b780002002000884d2000a4
:10a19c000e04440088047800820c7800970180003b
:10a1ac00694d20008e8444001904be000801d000c3
:10a1bc008401d000030241004220a80085824c009b
:10a1cc004200a9004220ae004200a8000482d30045
:10a1dc000503780096018800040278001442780088
:10a1ec00970188000440e800610ab800848fd2000f
:10a1fc008582d2000402780004f0a10008c025007a
:10a20c00a64d20000e03430086037800880b7800cf
:10a21c0002002000c94d20008e8444008900780083
:10a22c0082087800a74d20008e8343001703be00e0
:10a23c000604d0008404d000090244004220a80087
:10a24c0085824b004200a9004220ae004200a800cb
:10a25c000482d300a7018000050378000402780073
:10a26c00a6018800004a7800a701880054f020005d
:10a27c009e004200610ab800848fd2008582d20011
:10a28c000402780004f0a10006c02500e24d200075
:10a29c000e01410082017800860978000900200037
:10a2ac00074e20008e83430007047800090c7800c9
:10a2bc0097018000e34d20008e8141001301be0008
:10a2cc000203d0000404d000080243004220a8007e
:10a2dc00858249004200a9004220ae004200a8003d
:10a2ec000482d300050378009601880004027800ec
:10a2fc0014427800970188000440e800610ab80015
:10a30c00848fd2008582d2000402780004f0a10070
:10a31c0002c02500294e20008e844400890078005c
:10a32c008208780007002000434e20008e814100f7
:10a33c0003037800070b7800294e20008e8444001c
:10a34c001904be008800d0000401d0000282400035
:10a35c004220a80085824c004200a9004220ae0099
:10a36c004200a8000482d300a701800005037800f6
:10a37c0004027800a6018800004a7800a701880032
:10a38c0064f020009e004200610ab800848fd20065
:10a39c008582d2000402780004f0a10007c02500d9
:10a3ac00634e20008e81410003037800070b780078
:10a3bc0002002000884e20000e044400880478001f
:10a3cc00820c780097018000694e20008e84440036
:10a3dc001904be000801d0008401d0000302410022
:10a3ec004220a80085824c004200a9004220ae0009
:10a3fc004200a8000482d30005037800960188006f
:10a40c000402780014427800970188000440e800a8
:10a41c00610ab800848fd2008582d20004027800d1
:10a42c0004f0a10008c02500a64e20000e03430036
:10a43c0086037800880b780002002000c94e2000ab
:10a44c008e8444008900780082087800a74e200092
:10a45c008e8343001703be000604d0008404d00092
:10a46c00090244004220a80085824b004200a9004a
:10a47c004220ae004200a8000482d300a701800055
:10a48c000503780004027800a6018800004a7800d1
:10a49c00a701880014fa20009e004200610ab8004f
:10a4ac00848fd2008582d2000402780004f0a100cf
:10a4bc0006c02500e24e20000e014100820178000a
:10a4cc008609780009002000074f20008e83430086
:10a4dc0007047800090c780097018000e34e2000f7
:10a4ec008e8141001301be000203d0000404d00091
:10a4fc00080243004220a800858249004200a900be
:10a50c004220ae004200a8000482d300050378006c
:10a51c0096018800040278001442780097018800a4
:10a52c000440e800610ab800848fd2008582d20012
:10a53c000402780004f0a10002c02500294f20007d
:10a54c008e8444008900780082087800070020007f
:10a55c00434f20008e81410003037800070b7800e5
:10a56c00294f20008e8444001904be008800d000be
:10a57c000401d000028240004220a80085824c00d9
:10a58c004200a9004220ae004200a8000482d30081
:10a59c00a70180000503780004027800a60188005a
:10a5ac00004a7800a701880024fa20009e0042008f
:10a5bc00610ab800848fd2008582d2000402780030
:10a5cc0004f0a10007c02500634f20008e814100dc
:10a5dc0003037800070b780002002000884f20004e
:10a5ec000e04440088047800820c780097018000e7
:10a5fc00694f20008e8444001904be000801d0006d
:10a60c008401d000030241004220a80085824c0046
:10a61c004200a9004220ae004200a8000482d300f0
:10a62c000503780096018800040278001442780033
:10a63c00970188000440e800610ab800848fd200ba
:10a64c008582d2000402780004f0a10008c0250025
:10a65c00a64f20000e03430086037800880b780079
:10a66c0002002000c94f20008e844400890078002d
:10a67c0082087800a74f20008e8343001703be008a
:10a68c000604d0008404d000090244004220a80033
:10a69c0085824b004200a9004220ae004200a80077
:10a6ac000482d300a701800005037800040278001f
:10a6bc00a6018800004a7800a701880034fa20001f
:10a6cc009e004200610ab800848fd2008582d200bd
:10a6dc000402780004f0a10006c02500e24f20001f
:10a6ec000e014100820178008609780009002000e3
:10a6fc00075020008e83430007047800090c780073
:10a70c0097018000e34f20008e8141001301be00b1
:10a71c000203d0000404d000080243004220a80029
:10a72c00858249004200a9004220ae004200a800e8
:10a73c000482d30005037800960188000402780097
:10a74c0014427800970188000440e800610ab800c0
:10a75c00848fd2008582d2000402780004f0a1001c
:10a76c0002c02500295020008e8444008900780006
:10a77c008208780007002000435020008e814100a1
:10a78c0003037800070b7800295020008e844400c6
:10a79c001904be008800d0000401d00002824000e1
:10a7ac004220a80085824c004200a9004220ae0045
:10a7bc004200a8000482d300a701800005037800a2
:10a7cc0004027800a6018800004a7800a7018800de
:10a7dc0044fa20009e004200610ab800848fd20027
:10a7ec008582d2000402780004f0a10007c0250085
:10a7fc00635020008e81410003037800070b780022
:10a80c0002002000885020000e04440088047800c8
:10a81c00820c780097018000695020008e844400df
:10a82c001904be000801d0008401d00003024100cd
:10a83c004220a80085824c004200a9004220ae00b4
:10a84c004200a8000482d30005037800960188001a
:10a85c000402780014427800970188000440e80054
:10a86c00610ab800848fd2008582d200040278007d
:10a87c0004f0a10008c02500a65020000e034300e0
:10a88c0086037800880b780002002000c950200055
:10a89c008e8444008900780082087800a75020003c
:10a8ac008e8343001703be000604d0008404d0003e
:10a8bc00090244004220a80085824b004200a900f6
:10a8cc004220ae004200a8000482d300a701800001
:10a8dc000503780004027800a6018800004a78007d
:10a8ec00a701880054fa20009e004200610ab800bb
:10a8fc00848fd2008582d2000402780004f0a1007b
:10a90c0006c02500e25020000e01410082017800b3
:10a91c008609780009002000075120008e8343002f
:10a92c0007047800090c780097018000e3502000a0
:10a93c008e8141001301be000203d0000404d0003c
:10a94c00080243004220a800858249004200a90069
:10a95c004220ae004200a8000482d3000503780018
:10a96c009601880004027800144278009701880050
:10a97c000440e800610ab800848fd2008582d200be
:10a98c000402780004f0a10002c025002951200027
:10a99c008e8444008900780082087800070020002b
:10a9ac00435120008e81410003037800070b78008f
:10a9bc00295120008e8444001904be008800d00068
:10a9cc000401d000028240004220a80085824c0085
:10a9dc004200a9004220ae004200a8000482d3002d
:10a9ec00a70180000503780004027800a601880006
:10a9fc00004a7800a701880064fa20009e004200fb
:10aa0c00610ab800848fd2008582d20004027800db
:10aa1c0004f0a10007c02500635120008e81410085
:10aa2c0003037800070b78000200200088512000f7
:10aa3c000e04440088047800820c78009701800092
:10aa4c00695120008e8444001904be000801d00016
:10aa5c008401d000030241004220a80085824c00f2
:10aa6c004200a9004220ae004200a8000482d3009c
:10aa7c0005037800960188000402780014427800df
:10aa8c00970188000440e800610ab800848fd20066
:10aa9c008582d2000402780004f0a10008c02500d1
:10aaac00a65120000e03430086037800880b780023
:10aabc0002002000c95120008e84440089007800d7
:10aacc0082087800a75120008e8343001703be0034
:10aadc000604d0008404d000090244004220a800df
:10aaec0085824b004200a9004220ae004200a80023
:10aafc000482d300a70180000503780004027800cb
:10ab0c00a6018800004a7800a701880014042100df
:10ab1c009e004200610ab800848fd2008582d20068
:10ab2c000402780004f0a10006c02500e2512000c8
:10ab3c000e0141008201780086097800090020008e
:10ab4c00075220008e83430007047800090c78001c
:10ab5c0097018000e35120008e8141001301be005b
:10ab6c000203d0000404d000080243004220a800d5
:10ab7c00858249004200a9004220ae004200a80094
:10ab8c000482d30005037800960188000402780043
:10ab9c0014427800970188000440e800610ab8006c
:10abac00848fd2008582d2000402780004f0a100c8
:10abbc0002c02500295220008e84440089007800b0
:10abcc008208780007002000435220008e8141004b
:10abdc0003037800070b7800295220008e84440070
:10abec001904be008800d0000401d000028240008d
:10abfc004220a80085824c004200a9004220ae00f1
:10ac0c004200a8000482d300a7018000050378004d
:10ac1c0004027800a6018800004a7800a701880089
:10ac2c00240421009e004200610ab800848fd200e7
:10ac3c008582d2000402780004f0a10007c0250030
:10ac4c00635220008e81410003037800070b7800cb
:10ac5c0002002000885220000e0444008804780072
:10ac6c00820c780097018000695220008e84440089
:10ac7c001904be000801d0008401d0000302410079
:10ac8c004220a80085824c004200a9004220ae0060
:10ac9c004200a8000482d3000503780096018800c6
:10acac000402780014427800970188000440e80000
:10acbc00610ab800848fd2008582d2000402780029
:10accc0004f0a10008c02500a65220000e0343008a
:10acdc0086037800880b780002002000c9522000ff
:10acec008e8444008900780082087800a7522000e6
:10acfc008e8343001703be000604d0008404d000ea
:10ad0c00090244004220a80085824b004200a900a1
:10ad1c004220ae004200a8000482d300a7018000ac
:10ad2c000503780004027800a6018800004a780028
:10ad3c00a7018800340421009e004200610ab8007b
:10ad4c00848fd2008582d2000402780004f0a10026
:10ad5c0006c02500e25220000e014100820178005d
:10ad6c008609780009002000075320008e834300d9
:10ad7c0007047800090c780097018000e35220004a
:10ad8c008e8141001301be000203d0000404d000e8
:10ad9c00080243004220a800858249004200a90015
:10adac004220ae004200a8000482d30005037800c4
:10adbc0096018800040278001442780097018800fc
:10adcc000440e800610ab800848fd2008582d2006a
:10addc000402780004f0a10002c0250029532000d1
:10adec008e844400890078008208780007002000d7
:10adfc00435320008e81410003037800070b780039
:10ae0c00295320008e8444001904be008800d00011
:10ae1c000401d000028240004220a80085824c0030
:10ae2c004200a9004220ae004200a8000482d300d8
:10ae3c00a70180000503780004027800a6018800b1
:10ae4c00004a7800a7018800440421009e004200bb
:10ae5c00610ab800848fd2008582d2000402780087
:10ae6c0004f0a10007c02500635320008e8141002f
:10ae7c0003037800070b78000200200088532000a1
:10ae8c000e04440088047800820c7800970180003e
:10ae9c00695320008e8444001904be000801d000c0
:10aeac008401d000030241004220a80085824c009e
:10aebc004200a9004220ae004200a8000482d30048
:10aecc00050378009601880004027800144278008b
:10aedc00970188000440e800610ab800848fd20012
:10aeec008582d2000402780004f0a10008c025007d
:10aefc00a65320000e03430086037800880b7800cd
:10af0c0002002000c95320008e8444008900780080
:10af1c0082087800a75320008e8343001703be00dd
:10af2c000604d0008404d000090244004220a8008a
:10af3c0085824b004200a9004220ae004200a800ce
:10af4c000482d300a7018000050378000402780076
:10af5c00a6018800004a7800a7018800540421004b
:10af6c009e004200610ab800848fd2008582d20014
:10af7c000402780004f0a10006c02500e253200072
:10af8c000e0141008201780086097800090020003a
:10af9c00075420008e83430007047800090c7800c6
:10afac0097018000e35320008e8141001301be0005
:10afbc000203d0000404d000080243004220a80081
:10afcc00858249004200a9004220ae004200a80040
:10afdc000482d300050378009601880004027800ef
:10afec0014427800970188000440e800610ab80018
:10affc00848fd2008582d2000402780004f0a10074
:10b00c0002c02500295420008e8444008900780059
:10b01c008208780007002000435420008e814100f4
:10b02c0003037800070b7800295420008e84440019
:10b03c001904be008800d0000401d0000282400038
:10b04c004220a80085824c004200a9004220ae009c
:10b05c004200a8000482d300a701800005037800f9
:10b06c0004027800a6018800004a7800a701880035
:10b07c00640421009e004200610ab800848fd20053
:10b08c008582d2000402780004f0a10007c02500dc
:10b09c00635420008e81410003037800070b780075
:10b0ac0002002000885420000e044400880478001c
:10b0bc00820c780097018000695420008e84440033
:10b0cc001904be000801d0008401d0000302410025
:10b0dc004220a80085824c004200a9004220ae000c
:10b0ec004200a8000482d300050378009601880072
:10b0fc000402780014427800970188000440e800ac
:10b10c00610ab800848fd2008582d20004027800d4
:10b11c0004f0a10008c02500a65420000e03430033
:10b12c0086037800880b780002002000c9542000a8
:10b13c008e8444008900780082087800a75420008f
:10b14c008e8343001703be000604d0008404d00095
:10b15c00090244004220a80085824b004200a9004d
:10b16c004220ae004200a8000482d300a701800058
:10b17c000503780004027800a6018800004a7800d4
:10b18c00a7018800140e21009e004200610ab8003d
:10b19c00848fd2008582d2000402780004f0a100d2
:10b1ac0006c02500e25420000e0141008201780007
:10b1bc008609780009002000075520008e83430083
:10b1cc0007047800090c780097018000e3542000f4
:10b1dc008e8141001301be000203d0000404d00094
:10b1ec00080243004220a800858249004200a900c1
:10b1fc004220ae004200a8000482d3000503780070
:10b20c0096018800040278001442780097018800a7
:10b21c000440e800610ab800848fd2008582d20015
:10b22c000402780004f0a10002c02500295520007a
:10b23c008e84440089007800820878000700200082
:10b24c00435520008e81410003037800070b7800e2
:10b25c00295520008e8444001904be008800d000bb
:10b26c000401d000028240004220a80085824c00dc
:10b27c004200a9004220ae004200a8000482d30084
:10b28c00a70180000503780004027800a60188005d
:10b29c00004a7800a7018800240e21009e0042007d
:10b2ac00610ab800848fd2008582d2000402780033
:10b2bc0004f0a10007c02500635520008e814100d9
:10b2cc0003037800070b780002002000885520004b
:10b2dc000e04440088047800820c780097018000ea
:10b2ec00695520008e8444001904be000801d0006a
:10b2fc008401d000030241004220a80085824c004a
:10b30c004200a9004220ae004200a8000482d300f3
:10b31c000503780096018800040278001442780036
:10b32c00970188000440e800610ab800848fd200bd
:10b33c008582d2000402780004f0a10008c0250028
:10b34c00a65520000e03430086037800880b780076
:10b35c0002002000c95520008e844400890078002a
:10b36c0082087800a75520008e8343001703be0087
:10b37c000604d0008404d000090244004220a80036
:10b38c0085824b004200a9004220ae004200a8007a
:10b39c000482d300a7018000050378000402780022
:10b3ac00a6018800004a7800a7018800340e21000d
:10b3bc009e004200610ab800848fd2008582d200c0
:10b3cc000402780004f0a10006c02500e25520001c
:10b3dc000e014100820178008609780009002000e6
:10b3ec00075620008e83430007047800090c780070
:10b3fc0097018000e35520008e8141001301be00af
:10b40c000203d0000404d000080243004220a8002c
:10b41c00858249004200a9004220ae004200a800eb
:10b42c000482d3000503780096018800040278009a
:10b43c0014427800970188000440e800610ab800c3
:10b44c00848fd2008582d2000402780004f0a1001f
:10b45c0002c02500295620008e8444008900780003
:10b46c008208780007002000435620008e8141009e
:10b47c0003037800070b7800295620008e844400c3
:10b48c001904be008800d0000401d00002824000e4
:10b49c004220a80085824c004200a9004220ae0048
:10b4ac004200a8000482d300a701800005037800a5
:10b4bc0004027800a6018800004a7800a7018800e1
:10b4cc00440e21009e004200610ab800848fd20015
:10b4dc008582d2000402780004f0a10007c0250088
:10b4ec00635620008e81410003037800070b78001f
:10b4fc0002002000885620000e04440088047800c6
:10b50c00820c780097018000695620008e844400dc
:10b51c001904be000801d0008401d00003024100d0
:10b52c004220a80085824c004200a9004220ae00b7
:10b53c004200a8000482d30005037800960188001d
:10b54c000402780014427800970188000440e80057
:10b55c00610ab800848fd2008582d2000402780080
:10b56c0004f0a10008c02500a65620000e034300dd
:10b57c0086037800880b780002002000c956200052
:10b58c008e8444008900780082087800a756200039
:10b59c008e8343001703be000604d0008404d00041
:10b5ac00090244004220a80085824b004200a900f9
:10b5bc004220ae004200a8000482d300a701800004
:10b5cc000503780004027800a6018800004a780080
:10b5dc00a7018800540e21009e004200610ab800a9
:10b5ec00848fd2008582d2000402780004f0a1007e
:10b5fc0006c02500e25620000e01410082017800b1
:10b60c008609780009002000075720008e8343002c
:10b61c0007047800090c780097018000e35620009d
:10b62c008e8141001301be000203d0000404d0003f
:10b63c00080243004220a800858249004200a9006c
:10b64c004220ae004200a8000482d300050378001b
:10b65c009601880004027800144278009701880053
:10b66c000440e800610ab800848fd2008582d200c1
:10b67c000402780004f0a10002c025002957200024
:10b68c008e8444008900780082087800070020002e
:10b69c00435720008e81410003037800070b78008c
:10b6ac00295720008e8444001904be008800d00065
:10b6bc000401d000028240004220a80085824c0088
:10b6cc004200a9004220ae004200a8000482d30030
:10b6dc00a70180000503780004027800a601880009
:10b6ec00004a7800a7018800640e21009e004200e9
:10b6fc00610ab800848fd2008582d20004027800df
:10b70c0004f0a10007c02500635720008e81410082
:10b71c0003037800070b78000200200088572000f4
:10b72c000e04440088047800820c78009701800095
:10b73c00695720008e8444001904be000801d00013
:10b74c008401d000030241004220a80085824c00f5
:10b75c004200a9004220ae004200a8000482d3009f
:10b76c0005037800960188000402780014427800e2
:10b77c00970188000440e800610ab800848fd20069
:10b78c008582d2000402780004f0a10008c02500d4
:10b79c00a65720000e03430086037800880b780020
:10b7ac0002002000c95720008e84440089007800d4
:10b7bc0082087800a75720008e8343001703be0031
:10b7cc000604d0008404d000090244004220a800e2
:10b7dc0085824b004200a9004220ae004200a80026
:10b7ec000482d300a70180000503780004027800ce
:10b7fc00a6018800004a7800a701880024182100bf
:10b80c009e004200610ab800848fd2008582d2006b
:10b81c000402780004f0a10006c02500e2572000c5
:10b82c000e01410082017800860978000900200091
:10b83c00075820008e83430007047800090c780019
:10b84c0097018000e35720008e8141001301be0058
:10b85c000203d0000404d000080243004220a800d8
:10b86c00858249004200a9004220ae004200a80097
:10b87c000482d30005037800960188000402780046
:10b88c0014427800970188000440e800610ab8006f
:10b89c00848fd2008582d2000402780004f0a100cb
:10b8ac0002c02500295820008e84440089007800ad
:10b8bc008208780007002000435820008e81410048
:10b8cc0003037800070b7800295820008e8444006d
:10b8dc001904be008800d0000401d0000282400090
:10b8ec004220a80085824c004200a9004220ae00f4
:10b8fc004200a8000482d300a70180000503780051
:10b90c0004027800a6018800004a7800a70188008c
:10b91c00341821009e004200610ab800848fd200c6
:10b92c008582d2000402780004f0a10007c0250033
:10b93c00635820008e81410003037800070b7800c8
:10b94c0002002000885820000e044400880478006f
:10b95c00820c780097018000695820008e84440086
:10b96c001904be000801d0008401d000030241007c
:10b97c004220a80085824c004200a9004220ae0063
:10b98c004200a8000482d3000503780096018800c9
:10b99c000402780014427800970188000440e80003
:10b9ac00610ab800848fd2008582d200040278002c
:10b9bc0004f0a10008c02500a65820000e03430087
:10b9cc0086037800880b780002002000c9582000fc
:10b9dc008e8444008900780082087800a7582000e3
:10b9ec008e8343001703be000604d0008404d000ed
:10b9fc00090244004220a80085824b004200a900a5
:10ba0c004220ae004200a8000482d300a7018000af
:10ba1c000503780004027800a6018800004a78002b
:10ba2c00a7018800441821009e004200610ab8005a
:10ba3c00848fd2008582d2000402780004f0a10029
:10ba4c0006c02500e25820000e014100820178005a
:10ba5c008609780009002000075920008e834300d6
:10ba6c0007047800090c780097018000e358200047
:10ba7c008e8141001301be000203d0000404d000eb
:10ba8c00080243004220a800858249004200a90018
:10ba9c004220ae004200a8000482d30005037800c7
:10baac0096018800040278001442780097018800ff
:10babc000440e800610ab800848fd2008582d2006d
:10bacc000402780004f0a10002c0250029592000ce
:10badc008e844400890078008208780007002000da
:10baec00435920008e81410003037800070b780036
:10bafc00295920008e8444001904be008800d0000f
:10bb0c000401d000028240004220a80085824c0033
:10bb1c004200a9004220ae004200a8000482d300db
:10bb2c00a70180000503780004027800a6018800b4
:10bb3c00004a7800a7018800541821009e0042009a
:10bb4c00610ab800848fd2008582d200040278008a
:10bb5c0004f0a10007c02500635920008e8141002c
:10bb6c0003037800070b780002002000885920009e
:10bb7c000e04440088047800820c78009701800041
:10bb8c00695920008e8444001904be000801d000bd
:10bb9c008401d000030241004220a80085824c00a1
:10bbac004200a9004220ae004200a8000482d3004b
:10bbbc00050378009601880004027800144278008e
:10bbcc00970188000440e800610ab800848fd20015
:10bbdc008582d2000402780004f0a10008c0250080
:10bbec00a65920000e03430086037800880b7800ca
:10bbfc0002002000c95920008e844400890078007e
:10bc0c0082087800a75920008e8343001703be00da
:10bc1c000604d0008404d000090244004220a8008d
:10bc2c0085824b004200a9004220ae004200a800d1
:10bc3c000482d300a7018000050378000402780079
:10bc4c00a6018800004a7800a70188002422210060
:10bc5c009e004200610ab800848fd2008582d20017
:10bc6c000402780004f0a10006c02500e25920006f
:10bc7c000e0141008201780086097800090020003d
:10bc8c00075a20008e83430007047800090c7800c3
:10bc9c0097018000e35920008e8141001301be0002
:10bcac000203d0000404d000080243004220a80084
:10bcbc00858249004200a9004220ae004200a80043
:10bccc000482d300050378009601880004027800f2
:10bcdc0014427800970188000440e800610ab8001b
:10bcec00848fd2008582d2000402780004f0a10077
:10bcfc0002c02500295a20008e8444008900780057
:10bd0c008208780007002000435a20008e814100f1
:10bd1c0003037800070b7800295a20008e84440016
:10bd2c001904be008800d0000401d000028240003b
:10bd3c004220a80085824c004200a9004220ae009f
:10bd4c004200a8000482d300a701800005037800fc
:10bd5c0004027800a6018800004a7800a701880038
:10bd6c00342221009e004200610ab800848fd20068
:10bd7c008582d2000402780004f0a10007c02500df
:10bd8c00635a20008e81410003037800070b780072
:10bd9c0002002000885a20000e0444008804780019
:10bdac00820c780097018000695a20008e84440030
:10bdbc001904be000801d0008401d0000302410028
:10bdcc004220a80085824c004200a9004220ae000f
:10bddc004200a8000482d300050378009601880075
:10bdec000402780014427800970188000440e800af
:10bdfc00610ab800848fd2008582d20004027800d8
:10be0c0004f0a10008c02500a65a20000e03430030
:10be1c0086037800880b780002002000c95a2000a5
:10be2c008e8444008900780082087800a75a20008c
:10be3c008e8343001703be000604d0008404d00098
:10be4c00090244004220a80085824b004200a90050
:10be5c004220ae004200a8000482d300a70180005b
:10be6c000503780004027800a6018800004a7800d7
:10be7c00a7018800442221009e004200610ab800fc
:10be8c00848fd2008582d2000402780004f0a100d5
:10be9c0006c02500e25a20000e0141008201780004
:10beac008609780009002000075b20008e83430080
:10bebc0007047800090c780097018000e35a2000f1
:10becc008e8141001301be000203d0000404d00097
:10bedc00080243004220a800858249004200a900c4
:10beec004220ae004200a8000482d3000503780073
:10befc0096018800040278001442780097018800ab
:10bf0c000440e800610ab800848fd2008582d20018
:10bf1c000402780004f0a10002c02500295b200077
:10bf2c008e84440089007800820878000700200085
:10bf3c00435b20008e81410003037800070b7800df
:10bf4c00295b20008e8444001904be008800d000b8
:10bf5c000401d000028240004220a80085824c00df
:10bf6c004200a9004220ae004200a8000482d30087
:10bf7c00a70180000503780004027800a601880060
:10bf8c00004a7800a7018800542221009e0042003c
:10bf9c00610ab800848fd2008582d2000402780036
:10bfac0004f0a10007c02500635b20008e814100d6
:10bfbc0003037800070b780002002000885b200048
:10bfcc000e04440088047800820c780097018000ed
:10bfdc00695b20008e8444001904be000801d00067
:10bfec008401d000030241004220a80085824c004d
:10bffc004200a9004220ae004200a8000482d300f7
:10c00c000503780096018800040278001442780039
:10c01c00970188000440e800610ab800848fd200c0
:10c02c008582d2000402780004f0a10008c025002b
:10c03c00a65b20000e03430086037800880b780073
:10c04c0002002000c95b20008e8444008900780027
:10c05c0082087800a75b20008e8343001703be0084
:10c06c000604d0008404d000090244004220a80039
:10c07c0085824b004200a9004220ae004200a8007d
:10c08c000482d300a7018000050378000402780025
:10c09c00a6018800004a7800a7018800242c210002
:10c0ac009e004200610ab800848fd2008582d200c3
:10c0bc000402780004f0a10006c02500e25b200019
:10c0cc000e014100820178008609780009002000e9
:10c0dc00075c20008e83430007047800090c78006d
:10c0ec0097018000e35b20008e8141001301be00ac
:10c0fc000203d0000404d000080243004220a80030
:10c10c00858249004200a9004220ae004200a800ee
:10c11c000482d3000503780096018800040278009d
:10c12c0014427800970188000440e800610ab800c6
:10c13c00848fd2008582d2000402780004f0a10022
:10c14c0002c02500295c20008e8444008900780000
:10c15c008208780007002000435c20008e8141009b
:10c16c0003037800070b7800295c20008e844400c0
:10c17c001904be008800d0000401d00002824000e7
:10c18c004220a80085824c004200a9004220ae004b
:10c19c004200a8000482d300a701800005037800a8
:10c1ac0004027800a6018800004a7800a7018800e4
:10c1bc00342c21009e004200610ab800848fd2000a
:10c1cc008582d2000402780004f0a10007c025008b
:10c1dc00635c20008e81410003037800070b78001c
:10c1ec0002002000885c20000e04440088047800c3
:10c1fc00820c780097018000695c20008e844400da
:10c20c001904be000801d0008401d00003024100d3
:10c21c004220a80085824c004200a9004220ae00ba
:10c22c004200a8000482d300050378009601880020
:10c23c000402780014427800970188000440e8005a
:10c24c00610ab800848fd2008582d2000402780083
:10c25c0004f0a10008c02500a65c20000e034300da
:10c26c0086037800880b780002002000c95c20004f
:10c27c008e8444008900780082087800a75c200036
:10c28c008e8343001703be000604d0008404d00044
:10c29c00090244004220a80085824b004200a900fc
:10c2ac004220ae004200a8000482d300a701800007
:10c2bc000503780004027800a6018800004a780083
:10c2cc00a7018800442c21009e004200610ab8009e
:10c2dc00848fd2008582d2000402780004f0a10081
:10c2ec0006c02500e25c20000e01410082017800ae
:10c2fc008609780009002000075d20008e8343002a
:10c30c0007047800090c780097018000e35c20009a
:10c31c008e8141001301be000203d0000404d00042
:10c32c00080243004220a800858249004200a9006f
:10c33c004220ae004200a8000482d300050378001e
:10c34c009601880004027800144278009701880056
:10c35c000440e800610ab800848fd2008582d200c4
:10c36c000402780004f0a10002c02500295d200021
:10c37c008e84440089007800820878000700200031
:10c38c00435d20008e81410003037800070b780089
:10c39c00295d20008e8444001904be008800d00062
:10c3ac000401d000028240004220a80085824c008b
:10c3bc004200a9004220ae004200a8000482d30033
:10c3cc00a70180000503780004027800a60188000c
:10c3dc00004a7800a7018800542c21001e0042005e
:10c3ec006102b800848fd2008582d20004027800ea
:10c3fc0004f0a10007c02500635d20008e81410080
:10c40c0003037800070b780001002000885d2000f2
:10c41c000e04440088047800810c78009701800099
:10c42c00635d20008e8141001301be000203d00029
:10c43c000404d000080243004220a8008582490071
:10c44c004200a9004220ae004200a8000482d300a2
:10c45c0005037800960188000402780014427800e5
:10c46c00970188000443e8006102b800848fd20071
:10c47c008582d2000402780004f0a10002c02500dd
:10c48c00a95d20008e844400890078008208780021
:10c49c0008002000c35d20008e81410083037800da
:10c4ac00880b7800a35d20008e8141001301be0033
:10c4bc008203d0000404d000088243004220a8006c
:10c4cc00858249004200a9004220ae004200a8002b
:10c4dc000482d300a70180000500780004027800d4
:10c4ec00a0018800064a7800a70188003436210094
:10c4fc009e034200613ab800848fd2008582d2003c
:10c50c000402780004f0a10002c02500e95d2000bf
:10c51c008e8444008900780082087800080020008e
:10c52c00035e20008e81410003037800080b780025
:10c53c0096018000e35d20008e8141001301be0056
:10c54c000204d0008404d000090244004220a80058
:10c55c00858249004200a9004220ae004200a8009a
:10c56c000482d30005007800900188000402780052
:10c57c0014427800960188000443e800613ab80040
:10c58c00848fd2008582d2000402780004f0a100ce
:10c59c0003c02500215e20008e8040000101780040
:10c5ac000309780009002000475e20008e834300b9
:10c5bc0007047800090c7800235e20008e8141006e
:10c5cc001301be008203d0000404d0000882430093
:10c5dc004220a800858249004200a9004220ae00fa
:10c5ec004200a8000482d300a70180000500780057
:10c5fc0004027800a0018800064a7800a701880090
:10c60c00443621009e034200613ab800848fd20068
:10c61c008582d2000402780004f0a10002c025003b
:10c62c00695e20008e8444008900780082087800be
:10c63c0008002000835e20008e81410003037800f7
:10c64c00080b780096018000635e20008e8141000b
:10c65c001301be000204d0008404d000090244007f
:10c66c004220a800858249004200a9004220ae0069
:10c67c004200a8000482d3000500780090018800d5
:10c68c000402780014427800960188000443e80004
:10c69c00613ab800848fd2008582d20004027800ff
:10c6ac0004f0a10003c02500a15e20008e80400094
:10c6bc00010178000309780009002000c75e200002
:10c6cc008e83430007047800090c7800a35e2000d9
:10c6dc008e8141001301be008203d0000404d000ff
:10c6ec00088243004220a800858249004200a9002c
:10c6fc004220ae004200a8000482d300a7018000b3
:10c70c000500780004027800a0018800064a780031
:10c71c00a70188004f06be004f05be004f04be00a7
:10c72c000080fa00000006009400fa00889fbe000a
:10c73c008a9fbe008c9fbe0050879800618798002e
:10c74c0072879800038f9800148f98000002eb00fa
:10c75c00040f78000002eb00240798000002eb00a5
:10c76c0034079800b30037003e029000050020000b
:10c77c000400be0048d007000002be00b2fd20003d
:10c78c00930424000400be0098d007000002be00f1
:10c79c000406be006e829000cfa2de000400be0034
:10c7ac003ad007000002be000401be000c00be001f
:10c7bc00d9cf07000002be000400be00bfd00700a6
:10c7cc000002be0002002000032224000400be0070
:10c7dc0086d007000002be000200200003222400c5
:10c7ec000400be006fcf07000002be000400be00b4
:10c7fc000bd007000002be00040378003e0290003c
:10c80c00050020000402420085824a0007802000b7
:10c81c0007024200060a78003e0290000500200044
:10c82c000400be001cd007000002be00b2fd2000b8
:10c83c00930424000400be006cd007000002be006c
:10c84c000406be007e829000cfa2de000400be0073
:10c85c000ed007000002be000401be000c00be009a
:10c86c00adcf07000002be000400be0093d007004d
:10c87c000002be0002002000c32024000400be0001
:10c88c005ad007000002be0002002000c320240082
:10c89c000400be0043cf07000002be000400be002f
:10c8ac00dfcf07000002be00040378003e029000b8
:10c8bc00050020000402420085824a0007c02000c7
:10c8cc0007024200060a78003e0290000500200094
:10c8dc000400be00f0cf07000002be00b2fd200035
:10c8ec00930424000400be0040d007000002be00e8
:10c8fc000406be000e8a9000cfa2de000400be002b
:10c90c00e2cf07000002be000401be000c00be0016
:10c91c0081cf07000002be000400be0067d00700f4
:10c92c000002be0002002000032a24000400be0006
:10c93c002ed007000002be0002002000832c240031
:10c94c000400be0017cf07000002be000400be00aa
:10c95c00b3cf07000002be00040378003e02900033
:10c96c00050020000402420085824a0007002100d5
:10c97c0007024200060a78003e02900005002000e3
:10c98c000400be00c4cf07000002be00b2fd2000b0
:10c99c00930424000400be0014d007000002be0063
:10c9ac000406be001e8a9000cfa2de000400be006a
:10c9bc00b6cf07000002be000401be000c00be0092
:10c9cc0055cf07000002be000400be003bd007009c
:10c9dc000002be0002002000432b24000400be0015
:10c9ec0002d007000002be0002002000432b2400ee
:10c9fc000400be00ebce07000002be000400be0027
:10ca0c0087cf07000002be00040378003e029000ae
:10ca1c00050020000402420085824a0007402100e4
:10ca2c0007024200060a78003e0290000402e80069
:10ca3c0034079800be029000f41f2000848f52002f
:10ca4c0049ff36000002eb00240798000f00370066
:10ca5c002e029000050020000402420085824a004c
:10ca6c005e83900004024300140278008402780074
:10ca7c002e02900085007800040078007dd207001b
:10ca8c002e0290000402e80024079800ae029000e9
:10ca9c00f40f2000848f5200edff36000002eb00f3
:10caac0024079800320037002e0290004423dd004a
:10cabc002e029000050020000402420085824a00ec
:10cacc00ea03470004824300060a7800ae02900095
:10cadc0004ff2f0004aab9000402780006102000fd
:10caec00040343002e0290000500200004024200c3
:10cafc0085824a00a70420008e83430004824300f1
:10cb0c00060a78002e0290004423dd002e029000cd
:10cb1c00050020000402420085824a00a702200082
:10cb2c008e83430004824300060a7800ae02900014
:10cb3c0004ff2f0004aab90004027800061020009c
:10cb4c00040343002e029000050020000402420062
:10cb5c0085824a00a70620008e834300048243008e
:10cb6c00060a78002e0290000402e80024079800c0
:10cb7c002e029000ef0f5200cbff36000002eb00ac
:10cb8c0044079800af0037000002eb002407980020
:10cb9c009e0037002e029000050020000402420087
:10cbac0085824a006a03470004024300140278009d
:10cbbc008402e8006e829000040242001100090019
:10cbcc008482d80001027800040378002e029000c1
:10cbdc00050020000402420085824a00ea03470057
:10cbec0004824300060a78002e0290000500200003
:10cbfc000402420085824a00a60420000e03430072
:10cc0c0004024300140278008482e8007e829000c3
:10cc1c0004024200110009008482d800010278004d
:10cc2c00040378002e02900005002000040242004c
:10cc3c0085824a00a70420008e83430004824300af
:10cc4c00060a78002e029000050020000402420023
:10cc5c0085824a00a60220000e0343000402430012
:10cc6c00140278008402e8000e8a9000040242004c
:10cc7c00110009008482d8000102780004037800b6
:10cc8c002e029000050020000402420085824a001a
:10cc9c00a70220008e83430004824300060a78001a
:10ccac002e029000050020000402420085824a00fa
:10ccbc00a60620000e034300040243001402780071
:10cccc008482e8001e8a90000402420011000900d0
:10ccdc008482d80001027800040378002e029000b0
:10ccec00050020000402420085824a00a7062000ad
:10ccfc008e83430004824300060a78002e029000c3
:10cd0c00050020000402420085824a00a602200091
:10cd1c000e034300040243001402780005002000b7
:10cd2c000402420085824a000600210006024200ed
:10cd3c00140378002e02900005002000040242002b
:10cd4c0085824a00a70620008e834300048243009c
:10cd5c0014027800050020000402420085824a007b
:10cd6c00074021000702420014027800040f430020
:10cd7c009e027800040a200004aab900040278007c
:10cd8c00040f78002e0290000500200004024200df
:10cd9c0085824a006a0347000402430014027800ab
:10cdac00050020000402420085824a000680200013
:10cdbc0006024200140378002e02900005002000a9
:10cdcc000402420085824a00a70420008e8343009f
:10cddc000482430014027800050020000402420083
:10cdec0085824a0007c02000070242001402780026
:10cdfc00040243001e0f42001e007800b3d107004e
:10ce0c002e0290000402e800240798002e029000e5
:10ce1c00ef0f52005fff36000a87a90000000000e8
:10ce2c0001003700000000005438800070026200de
:10ce3c00e00f5200fbff32004e0290000402e800ab
:10ce4c0044079800ce029000f44a2000848f5200d0
:10ce5c004dff36000002eb00040f7800043c2f005d
:10ce6c00140798000002eb004407980058003700a4
:10ce7c000a87a90000000000010037000000000034
:10ce8c005438800070026200e00f5200fbff320049
:10ce9c000002eb00240798001c0037001e027800eb
:10ceac0005002000848fd2008582d2000402780015
:10cebc0004f0a10008c02500090020000043eb008d
:10cecc008803d0000400d000008243004220a80058
:10cedc0085824c004200a9004220ae004200a8000e
:10ceec000482d300a70180000500780004027800ba
:10cefc00a0018800064a7800a70188001e0fe800f0
:10cf0c002e0290000402e80024079800ae02900064
:10cf1c00f4092000848f5200e0ff36000002eb0081
:10cf2c00240798001e0037001e0290000402e9003e
:10cf3c00140798001e02900005002000848fd20078
:10cf4c008582d2000402780004f0a1000ac02500fa
:10cf5c000b0020000043eb008a00d0008403d000bb
:10cf6c00078240004220a80085824d004200a900a3
:10cf7c004220ae004200a8000482d300a70180002a
:10cf8c000500780004027800a0018800064a7800a9
:10cf9c00a70188002e0290000402e80024079800e4
:10cfac00ae029000f4092000848f5200deff3600a0
:10cfbc00000a20001e0f40001e029000040ab1005f
:10cfcc00140798004e0290000402e80044079800f1
:10cfdc00ce029000240c2000848f5200a4ff360057
:10cfec004f06be004f05be004f04be000080fa0085
:10cffc00000006000a00fa000003eb004607980048
:10d00c000003eb00160798005a0037001e0390002f
:10d01c006c33b90006037800360798004b003700d4
:10d02c000a87a90000000000010037000000000082
:10d03c005638800070036300e00f5300fbff320092
:10d04c000003eb00060f78003a0037001e03900037
:10d05c007433b900060378001e034300cfb3de001f
:10d06c0000e021000003430016437800e14f530019
:10d07c002f003a001e0378004333dd00260798008a
:10d08c00260037002e0390006130b900be039000db
:10d09c00060a200006bbb90006037800cfb3de00f9
:10d0ac000000430081804b004668200017002000e0
:10d0bc000003430081834b00868fd2008783d2000c
:10d0cc000603780006f0a10004c02500050020002e
:10d0dc00f0c3b3008400d0000601d00002834000ee
:10d0ec004220a80087834a004200a9004220ae00db
:10d0fc004200a8000683d300a1018000070178003c
:10d10c0006037800a2018800004b7800a10188007a
:10d11c002e0390000603e800260798001e03e80083
:10d12c00c333dd002e039000868f5300d5ff3c00e7
:10d13c001e0fe8001e037800f30f5300c3ff3400ea
:10d14c003e0390000603e800360798001e0390008b
:10d15c000603e8006c33b900860378003e039000a8
:10d16c00868f5300aeff3c001e0390000603e800c0
:10d17c00160798001e039000e40f5300a3ff340021
:10d18c000080fa00000006004a00fa006a0047001e
:10d19c00617d28001f000900311878000002eb00a7
:10d1ac00142788000002eb00242788000002eb0003
:10d1bc00342788000002eb00542788000002eb00a3
:10d1cc00642788000002eb004416880094cf070007
:10d1dc0000c025000100200038d007009bd00700bc
:10d1ec000887a80000c025000100200044d00700db
:10d1fc000002eb00040f78000b0037001e027800d1
:10d20c00cfa2de000402420085824a000680210083
:10d21c000602420014027800840078001e00780098
:10d22c0094d007001e0fe800f40f20009e02780037
:10d23c00848f5200f1ff34000002eb00040f7800e1
:10d24c00090037000a87a900000000000100370020
:10d25c00000000005438800070026200e00f5200a1
:10d26c00fbff32001e0fe800940f20009e02780096
:10d27c00848f5200f3ff34005eff07000002eb00c6
:10d28c00040f78001e027800cfa2de0004024200d8
:10d29c0085824a006a034700040243009402780026
:10d2ac00150798001e0fe8001e027800cfa2de00c2
:10d2bc000402420085824a006a03470004024300cc
:10d2cc0014007800200798001e0fe8001e0278005a
:10d2dc00cfa2de000402420085824a006a034700a6
:10d2ec000402430094007800310798001e0fe800f8
:10d2fc001e027800cfa2de000402420085824a00a2
:10d30c006a03470004024300940278004507980022
:10d31c001e0fe8009e027800040220001100090094
:10d32c008402d80001027800040f78004e029000ad
:10d33c00be0190002e0190009e0090000080210004
:10d34c00f9fc07001e027800cfa2de0004024200a6
:10d35c0085824a006a034700040243009402780065
:10d36c00150798001e0fe8001e027800cfa2de0001
:10d37c000402420085824a006a034700040243000b
:10d38c0014007800200798001e0fe8001e02780099
:10d39c00cfa2de000402420085824a006a034700e5
:10d3ac000402430094007800310798001e0fe80037
:10d3bc001e027800cfa2de000402420085824a00e1
:10d3cc006a03470004024300940278004507980062
:10d3dc001e0fe8009e0278000402200011000900d4
:10d3ec008402d80001027800040f78004e029000ed
:10d3fc00be0190002e0190009e00900000a0210024
:10d40c00c9fc07001e027800cfa2de000402420015
:10d41c0085824a006a0347000402430094027800a4
:10d42c00150798001e0fe8001e027800cfa2de0040
:10d43c000402420085824a006a034700040243004a
:10d44c0014007800200798001e0fe8001e027800d8
:10d45c00cfa2de000402420085824a006a03470024
:10d46c000402430094007800310798001e0fe80076
:10d47c001e027800cfa2de000402420085824a0020
:10d48c006a034700040243009402780045079800a1
:10d49c001e0fe8009e027800040220001100090013
:10d4ac008402d80001027800040f78004e0290002c
:10d4bc00be0190002e0190009e00900000c0210043
:08d4cc0099fc07006fff370017
:020000040000fa
:10d4d400005c0000002c0000800000000008000038
:10d4e4000010000080000000001800006406000026
:10d4f4008200000000002000004000006100810064
:10d5040000a10000c20002000123010043016300e6
:10d5140001840100a401c4000105020025024600a3
:10d52400026602008602a70002c702000803280060
:10d5340003490b006a0b8b0013ab1300cc1b0d00cb
:10d54400242e24004e2c6f002c903400b134d100d2
:10d554003c124500334554004d744d009555b600ba
:10d5640055d75d001866180066386e005976590064
:10d574007e7986009a8eba0096ba9e00dba6fb00de
:10d58400aefbae001cb73c00bf5dc7005dcf7d00a5
:10d59400d79edf009ee7be00efdff700fff7ff0036
:10d5a400ffffff00deffbd00f7bcf7009bf77a002a
:10d5b400ef59ef0058ef3700e716e70016e7f500dc
:10d5c400ded4de00b3d6b200d691d60070ce6f00a2
:10d5d400ce4ece002dc60d00c60cc600cbbdaa0093
:10d5e400b56ab50049ad0900ade8a400a8a4870058
:10d5f4009c4694002694e5008ba58b00848344000c
:10d6040083237b00e272c20072816a00616a200097
:10d6140062006200e059c00051a05100a04980009e
:10d624004960410040414000392031000031e000b0
:10d6340028e02800c020a00020801800801060008e
:10d644001040080020082000000000000000000036
:10d654000801080001100100100218000220030054
:10d664002003280003280400300430000438050097
:10d6740040054000064806004806500007500700d1
:10d684005808600028604900686a68008b70ab0025
:10d6940070cc78000d812e00814e89006f89900036
:10d6a40091b19100d1991200a233a20054aa74003e
:10d6b400aa95b200b6b2d700ba18c30038c378002e
:10d6c400c3b9cb00f9cb3900cc5ad4009ad4da00d0
:10d6d400d41bdd005bdd7b00ddbce500fce53d002b
:10d6e400ee7dee009deede00f61ef7005ef79f0075
:10d6f400ffbfff00ffffff00ffdeff00bdf7bc0020
:10d70400f79bf7007aef5900ef58ef0037e7160060
:10d71400e716e700f5ded400deb3d600b2d69100fa
:10d72400d670ce006fce4e00ce2dc6000dc60c00b6
:10d73400c6ebbd00aab58a00ad69ad0049a52800b5
:10d744009d089500e794a6008c868400657c4500be
:10d7540074247400046ce30063a25b00825b6100c8
:10d7640053414b002043000043e03a00a03a8000bc
:10d7740032603200403220002a002a00e029a00052
:10d784002180210060194000192019000011e000d7
:10d7940010a0100080086000084000002000000075
:10d7a4000000000001000100080208000208030054
:10d7b40010041000041805001805180006200600bf
:10d7c40020072000082808002809300009300a0032
:10d7d400300a38000b380c00402c40004d486d00d6
:10d7e400508e5800ae58cf0060106900307151005f
:10d7f400717179009281b20089d389001492340046
:10d804009a55a20075a29600aab6b200d7ba18001b
:10d81400c338c30078c3b900cbf9cb0039cc5a0064
:10d82400d49ad400dad41b00dd5bdd007bddbc00c0
:10d83400e5fce5003dee7d00ee9dee00def61e000b
:10d84400f75ef7009fffbf00ffffff00dfff9f00b1
:10d85400ff5ef7001ef7de00f6bdee007dee3d0034
:10d86400eefce500bce59c00e55bdd001bddda00b9
:10d87400d49ad4007ad43900ccf9cb00b9cb78004f
:10d88400c358c30018c3f700bab6b20096aa75000d
:10d89400aa55a200349a140092f39100b28992001e
:10d8a400817179005171300071106900ef60ae0030
:10d8b400588e58006d504d00482c40000c400b0011
:10d8c400380a38000a3009003009300008280800f6
:10d8d4002807280006200600200518000518040063
:10d8e40018041000031002001002080001080100cf
:10d8f4000000000000000000002100004100620060
:10d90400006200008300a40000c40000c500e5001c
:10d914000006010026012700014801006801890072
:10d9240001890100aa01ca0001eb01000c022c00cc
:10d93400026d0a008d0ace0012ee12002f1b500059
:10d9440023902300b12bf1002b12340052347300c6
:10d954003cb44400d44415004d354d007655960032
:10d9640055d75d001866180066386e005976590060
:10d974007e7986009a8eba0096ba9e00dba6fb00da
:10d98400aefbae001cb73c00bf5dc7005dcf7d00a1
:10d99400d79edf009ee7be00efdff700fff7ff0032
:10d9a400ffffff00dff7be00efbee7009edf7d0054
:10d9b400d75dcf005dc73c00bf1cb7001cb7fb00a0
:10d9c400aedba600ba9eba00969a8e0079867900dc
:10d9d4007e597600386e18006e186600d75db60062
:10d9e40055765500554d15004df44400b44493004c
:10d9f4003c5234003234f1002bb12b009023500000
:10da0400232f1b00ee12ce00128d0a006d0a2c008b
:10da1400020c0200eb01ca0001aa0100a90189005d
:10da24000168010048014700012601000601e500e4
:10da340000e50000c400a40000830000820062002e
:10da440000410000210020000000000020004000f0
:10da5400006100008100a10000c200000201230057
:10da6400014301006301840001a40100c401050015
:10da7400022502004602660002860200a702c700d1
:10da840002080300280b480013681b008823a80021
:10da94002bc93300094429004c495400695c8a00ad
:10daa40064aa6c00ca740a00852a8d004b956b0029
:10dab4009d8ba500abadcb00b50cc6000cc62d00ec
:10dac400c64ece004fce7000ce91d600b2d6b30073
:10dad400d6d4de00f5def500de16e70037e75800a1
:10dae400ef59ef007aef9b00f79cf700bdf7de00db
:10daf400fffeff00ffffff00ffdff700beefbe00e9
:10db0400e79edf007dd75d00cf5dc7003cbf1c00f2
:10db1400b71cb700fbaedb00a6ba9e00ba969a000b
:10db24008e798600797e590076386e00186e18005a
:10db340066b75d00765d36005df55c00955c54006b
:10db440054145400b353720053325300f1529100f1
:10db54004a504a00104aaf00496e49002e41ed0078
:10db6400408d40004c400c00400b38000a380a003d
:10db7400300930000930080028082800072806006a
:10db840020062000051805001804180004100300de
:10db9400100210000208010008010000000000004b
:10dba40000000000210041000062000062008300c8
:10dbb40000a40000c400c50000e500000601260022
:10dbc4000127010048016800018901008901aa00b8
:10dbd40001ca0100eb010c00020c0a000d122d0019
:10dbe4001a2e22002e2a4f0032504200704a710031
:10dbf40052715a00926292006a937200b482b40025
:10dc04008ad59200d59ad600a2f6aa00f7b21800d7
:10dc1400c338c30078c3b900cbf9cb0039cc5a0060
:10dc2400d49ad400dad41b00dd5bdd007bddbc00bc
:10dc3400e5fce5003dee7d00ee9dee00def61e0007
:10dc4400f75ef7009fffbf00ffffff00ffffde004e
:10dc5400ffbdf700bcf79b00f77aef0059ef5800bf
:10dc6400ef37e70016e71600e7f5de00d4deb30071
:10dc7400d6b2d60091d67000ce6fce004ece2d0017
:10dc8400c60dc6000cc6ab00bd6bb5002bb5eb00d2
:10dc9400ac8bac004aa40a00a4aa9b006a932a0095
:10dca40093ea8a00898a490082098200a979690075
:10dcb40071287100e86888006848600008600700ff
:10dcc4005807500006500600480648000540050065
:10dcd4004005380004300400300328000328030002
:10dce40020022000021802001001100001080000a8
:10dcf4000800000000010100010001000101000012
:10dd04000100010001010000010101000000000008
:10dd140001000000000100000100010000010000fa
:10dd240001000000000000000000010000000000ed
:10dd340001000100000100000100010000010100d8
:10dd440001000000000100000000010000010000cb
:10dd540001000100000100000000000000000000bc
:10dd640001010100000101000100010000010000a7
:10dd7400010001000101000000000000641e000019
:0cdd840002000000800000000000000011
:020000040000fa
:10dd9000f03fb1000180b10006003500ee0309003c
:10dda00000000000403fb1000180b100fbff3d00da
:10ddb0001000b000203fb0000200350000800900d4
:08ddc000000000000000060055
:020000040000fa
:020000040005f5
:0457f400ffec0000c6
:020000040000fa
:020000040005f5
:0457f800be9b000054
:020000040000fa
:020000040005f5
:0457fc007f3f0000eb
:00000001FF
